:20000000003A0120093F020039FB021039FB021039FB021039FB021039FB021039FB021097
:1C00200039FB021039FB021039FB021039FB021039FB021039FB021011FB021002
:20003C002DE9F04F99B0054680780224532800F2C485DFE810F054009900A800B800C8000B
:20005C00DA00EA000C011B01C2052A0138015901C205C205C205C205C205C205C205C205DA
:20007C00C205C205C205C205C205C205C205C205C205C205C205650188019401A001AB0106
:20009C00BA01D401EB0107023A02C205C205C205C205C205C205600276028C02A202B80213
:2000BC00CD02DE020303C205C205C205C205C205C20538034C036003C2056D037703940390
:2000DC009D03A903B503C403CE03F1030E04310439044B045804640488048F049204EC1C20
:2000FC00E97A2A7B002320461CF066FD8DF8180006AB65200021012220F0D8FEDFF8100BF5
:20011C000078012800F25885204627F06FFD002800F0528505460079012840F04D8527F075
:20013C00F7FA00274FF400018DF83F008DF83800000ACDF83A108DF841708DF83E708DF8BF
:20015C0040008DF839000EAE214606F10A0027F0CBFD297815223346017069788770417037
:20017C004520FF2100F026BD27F064FD6979AA790023002423F04AFC8DF838000EAB6520F3
:20019C00012100F050BC27F005FB27F071FC01460EA8022227F002FD8DF8180006AB652080
:2001BC00022100F040BC27F0F5FA27F061FC01460EA8032227F0F2FC8DF8180006AB6520A0
:2001DC00032100F030BC27F0E5FA27F051FCEA7901460EA80023002425F0ECF98DF818006B
:2001FC0006AB6520042100F01EBC27F0D3FA27F03FFC01460EA8052227F0D0FC8DF81800E4
:20021C0006AB6520052100F00EBC0020DFF8284A27F0ACF9ADF85800681DA0478046E81D53
:20023C00A04795F809B0824605F10A07BBF1100F00F2AB830EAC5E46002E00F0A983384695
:20025C0027F092FD24F8020B013E0237F4E727F0A1FA27F00DFC01460EA8102227F09EFCAE
:20027C008DF8180006AB65200721DCE327F092FA27F0FEFB01460EA8112227F08FFC8DF89E
:20029C00180006AB65200821CDE327F0D3FC6A7B691D0023002422F0BBF98DF838000EAB47
:2002BC0065200A21BFE302208DF8200027F0C2FCADF81800681D27F057FDEA79064605F1E2
:2002DC0008018DF838200EAF781C27F02FF806A831463A46002300241EF0CAFF8DF85800ED
:2002FC0016AB65200B219EE327F0A4FC0021002421F074FC8DF838000EAB65200C2192E3D5
:20031C000020DFF8344927F031F9ADF85800681DA047804695F80F9005F11000A04705F1CE
:20033C001304AD7C83460F2D00F244830EAE2F46002F00F04283204627F016FD26F8020BD3
:20035C00013F0234F4E727F025FA27F016F926F0DDFF40F0438306A827F0C6FC43E327F028
:20037C0019FA27F00AF926F0D1FF40F04A8306A827F0BAFC4AE327F05DFC27F047FB8DF85B
:20039C0038000EAB6520232100F013BCDFF88018C8208DF81800E81C0978002900F07E8335
:2003BC0026F02FFC8DF81800A0E36879EE1CFE280BD12878082808D3A879FF2805D1304694
:2003DC0027F0D2FC314623F0C1FD0EA9304626F0F7F8002800F08E83054600249CE3E81C87
:2003FC00042124F0FBFAE97927F0E0FCDFF83C188DF83800022026F037FDDFF834180320C4
:20041C0026F032FD0EAB65202621D2E327F00CFC044605F10E0027F0A7FC297C6A7C034646
:20043C00E878CDE90012AA1D214624F003F8DFF8F8178DF83800042026F016FD0EAB65200D
:20045C002721B6E34FF00208E81C8DF8408027F08BFCADF8380068798DF85800A81D27F0F8
:20047C0083FC2E7A044600270935CDE9005716A80EA9224633461FF057FD27F0AFF910D124
:20049C00DFF888078DF84080CDE9005722463346C08AADF8380016A80EA91FF045FD8DF835
:2004BC00180006AB6520282183E30226E81C8DF8406027F059FC27F0DBFAED7904460EA814
:2004DC00002321462A4625F055FF27F087F90ED1DFF838078DF8406021462A460023C08AA8
:2004FC00ADF838000EA825F045FF8DF8180006AB652029215DE327F04DF9ADF83800681DD8
:20051C00042124F06BFA6A7AAB7A0024014600940EA823F0BBFF8DF8180006AB6520302172
:20053C0081E227F037F927F076FA312201238DF8580016A8CDE90004DFF8E8060EA91FF017
:20055C00F3FC8DF8180006AB652031216BE227F021F927F060FA322201238DF8580016A869
:20057C00CDE90004DFF8BC060EA91FF0DDFC8DF8180006AB6520322155E227F00BF927F0DE
:20059C004AFA332201238DF8580016A8CDE90004DFF890060EA91FF0C7FC8DF8180006ABE9
:2005BC00652033213FE227F0F5F8ADF83800687B0024691D0094C0F3400200F001030EA884
:2005DC0021F0EEFA8DF8180006AB652034212AE227F0E0F86A7BADF83800691D0EA80023C2
:2005FC00002424F0E5FB8DF8180006AB6520352119E22C4614F8030B04281ABFE8782C1D69
:20061C0002208DF84000204627F0AEFBDFF81066A5780121E278ADF8380000230024317006
:20063C000EA829461DF0C0FB8DF818002846347024F0FAFB06AB65203621F4E127F0FAFA8C
:20065C00ADF83800687904218DF84000A81D24F0C5F90446AE7AEF7A05F10C0027F084FBCC
:20067C00DFF8A8850546214632463B4626F05BFF0EA81FF035FC27F0B1F810D1022021461F
:20069C0032463B468DF84000B8F81600ADF8380026F049FF0EA81FF023FC8DF8180006AB4D
:2006BC006520372185E26C7827F0C4FA0146DFF86C0500781FF0F0FB8DF8380004F0E0008F
:2006DC00202840F079820EAB65203E2171E26C7827F0B0FA0146DFF84405007820F0A6F869
:2006FC008DF8380004F0E000202840F065820EAB65203F215DE200206C788DF83800DFF879
:20071C0010050078411E022980F09181022092E127F090FA27F07AF98DF838000EAB652069
:20073C00422146E200200690ADF83C000E90E81C06A925F0EAF88DF83800069850B126F0C1
:20075C00F9FE81788DF83B10C1788DF83C1000798DF83D000EAB6520432106222AE2E81C9E
:20077C0026F04FFA8DF838000EAB6520442120E227F060FA6979AA790DF002FB8DF838006F
:20079C000EAB6520452114E227F054FA6979AA7919F072FB8DF838000EAB6520462108E277
:2007BC00EC7827F041FA0146204621F0ADFAB0FA80F0472140098DF838000EABBFE1E878C1
:2007DC0000248DF8384021F077FF0EAB6520472129E1E8780EA924F011FF06468DF8180081
:2007FC0040000130C5B2284627F0C2FA002800F0A181044600F8016B00219DF8182091420B
:20081C0080F0BC809DF83830013100F8023B9DF8393000F8013CF2E70EAC1321204626F036
:20083C0041FCEE7827F000FA0146304624F024FB002800F086810021231D8DF8381026F095
:20085C0079FEC11C827818468DF83B2026F06EFD7AE1002012218DF818000EAE304626F0DC
:20087C0021FCEC7827F0E0F9AA79ADF838000F2A28BF0F228DF83A201AB1F01CE91D26F0C8
:20089C0055FD0EA9204601221BF036FD8DF8180006AB65204B218CE126F040FB8DF83800B2
:2008BC000EAB65204C2184E1E87829798DF838100EA9032800F05F81022800F06281012865
:2008DC0040F0668152201FF0F5FF64E127F0B2F969790246A81D1AF0C5F88DF838000EAB3D
:2008FC0065204E2165E127F0A5F90146687918F0B9FE8DF838000EAB65204F2159E1C34D51
:20091C000822E88A05F13901ADF83800C14800788DF83A00A88CADF83B00688BADF83D00E9
:20093C000EACE01D26F002FD04F10F0005F11C01082226F0FBFC287E5021182223468DF842
:20095C004F00652036E1B2480078002800F0018112200AE11FF0ECF92EE100208DF8380087
:20097C00E878010606D5A94910F07F0018BF012081F868000EAB652053211AE16520492133
:20099C002A46234620F092FA39E180208DF863003E78102E52D80DF11809013734464D46A2
:2009BC00002C4DD0384627F0DFF925F8020B013C0237F5E780208DF8630027780F2F54D858
:2009DC0001340DF1180A3E46002E50D0204627F0CBF92AF8020B013E0234F5E7084627F0AE
:2009FC00C3F9ADF81800687E06A926F097FC0EA921201AF069FA8DF8580016AB652021215A
:200A1C0011E0084627F0B0F9ADF81800687E06A926F084FC0EA922201AF056FA8DF85800A3
:200A3C0016AB65202221012220F040FAC5E0002840F0B580042008F067FAB3E080200DE0D5
:200A5C00BBF1100F0CD80EA9002052465B468DE84202039016A8414613F0A0FB8DF86300A4
:200A7C000DF1630365200621A3E080200FE00F2D0FD80EA9002002974A465B46CDE900516D
:200A9C0006A9CDE9031016A8414614F071F88DF863000DF16303652020218AE016A90EAD1A
:200ABC002A4617F08BFD04469DF85800F0B1614904EB4400002641F8206001EB8000466075
:200ADC009DF94B00B0F1FF3F03DC05F1130021F06FFB0EAD1421284626F0E4FA04202146FA
:200AFC0014222B4623F0E2FE8DF8186006AB652024215EE0182027F03BF9002800F08380EC
:200B1C000446BDF8380000211822234626F09CFA0546002818BFC825192027F029F9002841
:200B3C0067D007460130002D4BD01821FF2226F0B3FA50E0002049218DF8180006AB6520F2
:200B5C0037E001208DF838000EAB65204A21132230E027F06FF8044605F10D0027F004F9B7
:200B7C000246691D204623F0A7FC8DF838000EAB652051211DE052201FF09CFE264800215B
:200B9C0004E052201FF096FE23480121017002E0522023F0E9FC0EAB65204D2109E0012040
:200BBC008DF8380004F0E000202805D10EAB65204021012220F07AF90024204619B0BDE82D
:200BDC00F08F3146082226F0B1FB07F109002146102226F0ABFB6520252119223B463D708D
:200BFC0020F064F93846192126F05CFA384627F0BDF8002CE0D02046182126F053FA2046BA
:200C1C0027F0B4F8D8E7C825FFF7E7BB48DD0020A80C00207C0A0020C30E0020B8E8002041
:200C3C00820E00200C0D0020654C0200615102004940010050A30020857D02002DE9F04F52
:200C5C0099B081466FF00700DFF8DC880630ADF8520098F80000022814D1DFF8C8080078DC
:200C7C0080B9B9F8080010B11020012101E03020002109F09DFF00208DF81C0007A9522089
:200C9C001FF018FE0DF11C0A99F80810D9F8040052460FF031FBE8B19DF81E709DF81F40FE
:200CBC009DF82050BDF8266026F02CFD844211D145EA070001280DD826F003004FF6F875E2
:200CDC0080B2A84206D098F80000022808D19DF84D0028B1D32014F0A8FD19B0BDE8F08F2F
:200CFC00B9F82800ADF84800B9F83200ADF82A009DF82200D0B1D9F804109DF81D209DF8DC
:200D1C003830012025F0D4FA08B1CF20E3E7DFF81C08C078012809D1B9F8280026F002FFB3
:200D3C0020B1417901F0E701083141719DF8210068B1BDF82610FF2024F09EF89DF82110FF
:200D5C00E0B141F001012C268DF8211017E09DF83900002800F005819DF83D10FF2902D06C
:200D7C00002940F02A81DFF8C807BDF82620C18A8A4240F02B810120222607E0082601F050
:200D9C000300012808BF46F01106012098F800103746022938BF67F07F07B20748BF37467D
:200DBC00002808BF37469DF82200002800F0818017F0400B1ED0012905D8DFF87407807B47
:200DDC00800700F1E780119801780C2900F2E880012241F298438A401A4200F0E180032993
:200DFC0002D140780D2805D007A821F024FE01283FF473AFDFF83847B9F84410A08C814298
:200E1C000AD199F84620B9F84210B9F8280000230093002307F008FC9DF82200F8B1B9F823
:200E3C004210B9F8280021F041F8002800F082800646D9F804009DF81D10F2780844417BB2
:200E5C008A421EBF00227260F1700130042123F0C5FD71688842FFF440AF0130706098F837
:200E7C00000002283ED2A07B80077FF536AF9DF84D0060B1BDF8280025F020FC002800F008
:200E9C001681D9F80400417801F0DF0141709DF82E00002800F0EE80D9F80400817901393D
:200EBC0081718DF82E1007F07F00090640F0E580E2E0DFF87C06C07A00283FF479AF07F078
:200EDC00220022283FF474AFF8B200F0420042287FF41BAF1198007800F0FE0006287FF401
:200EFC0014AF65E77FF4F9AE94F82600092802D004287FF4F2AEF8B2800600F18980BBF1E3
:200F1C00000F3FF4EAAE11980078033809283FF6E4AEDFE810F057010F010A000A005C01E7
:200F3C000A000A000A000A000B00D6E607A814F02DFBD2E69DF84D0000284ED0042024F0B3
:200F5C003DFA00283FF4C9AE01464FF4B2700880B9F828004880DFF8DC0500781CF0C4FD9A
:200F7C00BBE6BDF826001FF0E1FF0238DFF8C015B0FA80F0CA8A4109BDF82600904208BFD8
:200F9C000231002942D09DF81E20002A5AD001F1400759E0119801784A1E0B2AFFF41FAFAE
:200FBC00DFF88C05BDF82620C08A82427FF492AEBDF8280022F0C2FB8CE6109A9DF83C0058
:200FDC001FF068FB30B101200026DFE690F826000428F8D100260020D8E694F86C000128CE
:200FFC007FF43DAFBBF1000F04D01198007806283FF435AFE81DBDF82A1080B281423FF465
:20101C006CAE07A849461DF05BF866E600271BE099F8460026F072FA9DF82E00012840F019
:20103C00CA80B9F82800BDF82810814240F0C380BDF826001FF07AFF022804BF00208DF859
:20105C002E00B8E001F120071FF070FF0138B0FA80F0400947EA00069DF81E0000283FF436
:20107C0094AE1198007825F065FB012818BF07F07E068AE607F07F000746390702D44FF079
:20109C00000B34E0F9B24A0722D4C9069DF8211028D5C1F3820212B1072A18BF013A002A29
:2010BC0008BF074601F0E30040EA820118E0D32014F0BBFBDFF880040078002800F0A380CC
:2010DC00DFF8781451F82000C0EB001081009CE09DF8210000F0E00100F0E30040EAD1011A
:2010FC008DF82110D9F804004FF4805B017294F82600092801D0042826D1E18ABDF826009B
:20111C0088420AD01FF012FF022806D09DF8210000F0030001287FF4E0AD9DF81E00002842
:20113C0045D01198007803284CD007284FD004287FF4D3AD9DF8380002287FF4CEAD07A914
:20115C00002011F0B3FAC8E5FEB217F0610F47D0F00708D0B9F8281007A814F0B9FB002873
:20117C0066D007F09F074FF00008FEB2B80609D599F84600D9F83C2026F0C0F907A815A9AD
:20119C0005F076F9700640F14B81B9F8281007A80DF1520243460FF02BF900286FD0804699
:2011BC0011980078012808BF4BF0100B38E199F8460026F0A3F9D9F83C2007A815A905F07B
:2011DC0057F98AE507A800210EF09EFD85E59DF8380004287FF481AD07A816F0F3FD7CE5C1
:2011FC009DF81E0001285AD111980078032849D0052854D1B9F8281007A80DF15202002308
:20121C000FF0F6F869E5CD480168CD480268BDF82800904701287FF460ADCA480168BDF8ED
:20123C0028008847C8480168BDF82800884754E524F084FC9DF82E108046BDF8280019B961
:20125C00B9F82810884290D0E18A814204D1B748807801287FF489AFB9F8281007A8424671
:20127C0008F0F4FC002800F0C18030074BF0040BBDF8260048BFE81DADF8520075E74FF017
:20129C000008CDE0BDF8260025F018FA38B1B9F8281007A80DF1520200230FF0A9F89DF850
:2012BC002E0098B322F076F800287FF416AD9DF83900B0B3109A9DF83C009DF83D101FF01E
:2012DC00E9F9002800F095809DF83D00002800F09A80109926F0F4FB9DF82430ADF8520051
:2012FC0011209DF823209DF821104BF0400B002B08BF0920002A18BF0830002918BF0130F8
:20131C00D9F804100A5C013A0A5486E09DF81E0001287FF476AE1198007803283FF4DDACEC
:20133C006FE6BDF826003107ADF8520025D49DF8201011BB9DF81E1001291ED0002117F0A5
:20135C00D7FD18B140790138022816D3B9F84410BDF8520020F0AAFD28B1807824F01EFE0B
:20137C000138072809D3BDF8280025F0A7F9002800F0D18004208DF820004020BDF82610FE
:20139C000AF11D0200EAC7049DF82000234617F0E3FA38B1D9F804004BF0200B017801F0D2
:2013BC003F0101709DF8390048B1BDF826100AF1200020F0ABFA4BF0400BADF852009DF8CC
:2013DC001E00012806D0BDF82810BDF82600002213F02EFEBDF82810BDF82600224611F08A
:2013FC00D3FB002818BF4BF0200B16E007F0DF07B9E6BDF82610BDF828000B22002319F00B
:20141C00BFFAFFF76ABCBDF82600ADF8520026F089FB002808BF4BF0400B24F08FFB804696
:20143C00A81DBDF8521080B20E1A484818BF4646007801282BD1E81DB9F8321080B28142DD
:20145C0025D0B9F82810814221D0681CBDF8262080B282421BD2BDF82800814217D026F0DF
:20147C0061FBA0B101790139012910D8408801218DF85410ADF8600015AD28461DF066FA68
:20149C0028B1281D1CF054FA08B120F011FB78B2B0F1FF3F3FF721AC002E3FF41EACB9F8FB
:2014BC00080026F065FC00283FF417ACB9F80820D9F80410054625F039FF9DF81E1000203A
:2014DC0099F80830B9F8282016908DF85410BDF8521015ACCDE9006BCDE90204284610F07C
:2014FC003DF920B1284626F041FCFFF7F6BB0F48407800283FF4F1AB00208DF81860ADF899
:20151C001900DDF826004FEA3040059005A825F091FDFFF7E2BBBDF82610BDF8280002228E
:20153C006CE700BFC30E0020A80C0020600C002048DD0020BAE80020B50E00206892020046
:20155C00EC090020F4090020F0090020C10E00202DE9F0438DB0054680780224252800F207
:20157C007380DFE810F02600A100C100D400E700F5000301B602B6021C012D01B602B6022E
:20159C00B602B602B60245014A01B602B602530157016001B602B602B602B602B602B602A9
:2015BC00B602B602B6026A016D017001730177017E01DFF8D47500240E258DF80440387842
:2015DC00012807D801A81BF093FD04469DF8040005EB4005EEB2304626F0CAFB002800F082
:2015FC0087824FF000080546431C0021082280F80080012025F028FD26F08AF86872000ABB
:20161C000721A872DFF88405E972007828733878012800F262829DF80420002A6A7300F03F
:20163C005E8205F10E0000212346914280F0578213F8022B013100F8022B13F8012C00F845
:20165C00012C9DF80420F0E7A0F140010D291CD8DFE811F00E000F013F023F021D012D0101
:20167C003F023F02390144014F0164013F02730101ACE91C0822201D25F058FE204619F0F0
:20169C009BFABDF806004021EDE0632800F06C81642800F07981E02840F01B820024472072
:2016BC00E0210022002312E2202026F061FB002800F0C4812021FF22044625F0EDFC631C9C
:2016DC0001200021082225F0BFFC0546002818BF012501AB84200021042225F0B5FC0028BD
:2016FC0000F00882023509E2E81C26F03DFBADF80400832026F062FA014601AA832026F077
:20171C0021F98DF828000AAB6720022193E1E81C042123F063F90190842026F04FFA0146A0
:20173C0001AA842026F00EF98DF828000AAB6720032180E1612026F041FA0146EA1C612013
:20175C0026F000F98DF8040001AB6720042172E1622026F033FA0146EA1C622026F0F2F896
:20177C008DF8040001AB6720052164E100208DF80400E81C26F0F8FA6A7900F4F851002A27
:20179C0000F04C81B1F5A06F04D04FF6FF71884240F04E81DFF8EC034FF0FF3147E126F0F6
:2017BC00AFFA044625F078FFD949604301ACB0FBF1F1204626F04AFA672009210422ABE06D
:2017DC00DFF8B4632D79306840B901AC204625F072FE012021460DF05BFC3060052D00F0A2
:2017FC006A81002D00F06A81642120F035FD67E115F8032B672010216EE0E87820F00CFE10
:20181C008DF8040001AB6720112114E100246720142102E0002467201521ADF808400194A4
:20183C0001AB062253E100246720162109228DF80C40CDE9014401AB49E1F52020210BE094
:20185C00F520212108E0F520222105E04FF6F570232108E0F52024218DF8040001AB672004
:20187C00E9E0F5202521ADF828000AAB67200222E2E0E81C26F078FAADF8060001AC2046EF
:20189C0016F05CFA231D672041210822D4E0E81C0AA924F095FE00288DF8040000F0D0807A
:2018BC0001A81821FF22013025F0F6FBF5E0E81C0AA924F085FE00288DF8040000F0F2809C
:2018DC004FF0FF30F0E015F8030F697820F0A8FC28806720482102222B46ADE0E87823F0CD
:2018FC0077F901AC0146204617F0C2FC6720492111E0EC1C204624F09FFB002818BF2046DA
:20191C00B5F80B1018F0D8F801AC0146204617F0AFFC67204A21242223468DE001ACE91C3F
:20193C000822204625F002FD204625F0B1FA8DF828000AAB67204B217DE04FF0FF3095F814
:20195C000380691D0190ADF81000CDE902004FF6FE70ADF80600287903288DF8300020D194
:20197C000AA826F0C1F921E00024E91C08228DF8284001AD284625F0D9FC28461BF0D8FF32
:20199C000AAB67206321A1E0B5F80B006A7B0024E91C8DF8044009F07BFA01AB6720642135
:2019BC0094E0084626F0E0F9ADF82800AF7B002F00F0DD807E0095F80D90304626F0D8F9E2
:2019DC00002800F0D48005F10F013246044625F0ADFC00940AA940464A463B460CF0A6F881
:2019FC00002800F0BA80837801784278057946798DF806308DF804108DF80520C3788DF850
:201A1C0009608DF808508DF8073001A98B1D811D40794200184625F089FCA5E0B1F5A06F8B
:201A3C0003D04FF6FF71884202D156480021016001AB6720062101221FF038FA002448E03B
:201A5C00182026F095F940B3BDF828100446009006200022182322F013FFB8B9BDF828508F
:201A7C0001AE21461022701C25F060FC444F05EB450506F1110057F8251026F0E7F807EBC5
:201A9C008500416806F1150026F0E0F82046182125F008FB204626F069F901AB67204421D5
:201ABC001922C9E7BDF82800ADF8050001AB672045210322C0E7314901220A701FF0F5FD1B
:201ADC00002467200A218DF8044001AB01221FF0EDF920460DB0BDE8F08385F80D806720BB
:201AFC00002132462B461FF0E1F9284626F03EF97CBBA3E7019800BAC4F809000AAB8320EB
:201B1C000021022225F0A0FA20B1043506E000BF40420F00BDF82800A4F80D0004F10F03E8
:201B3C0061200021012225F08FFA002818BF083504F1100362200021102225F085FA002851
:201B5C0018BF1035234625706720012120221FF0ADF9204626F00AF970E74FF6FF70ADF880
:201B7C0008006FF480300190204626F0FFF801AB67204D210E225FE750E800207F0E00200E
:201B9C00A8E3002030E80020A80C00207C0A00202DE9F04F85B084780226362C00F2D28276
:201BBC000546DFE814F077017F01750087017B00CF02CF02840037004C008F00A200B000F9
:201BDC00CF02B8009B01CF02CF02A501B801C601CF02CF02CF02CF02CF02CF02CF0237000E
:201BFC004C00CF02CF02CF02CF02CF02CF02CF02CF02CF02CF02CF02CF02CF02CF02CF023E
:201C1C00CF02CF02CF02C000EE00D60102015B005B00E60126F002F8242840F0B58102ABA1
:201C3C00352000210422002425F00EFA002800F01282012002228DF81000002012E20020F1
:201C5C008DF8100025F0EAFF0646092C40F0F88095F8059095F806800720FAE0DFF81C750E
:201C7C0001208DF81000386880B1406A70B102A925F0DDFF0546342C40F03C82284626F03D
:201C9C0073F8002800F03582042052E2032050E2DFF8F834612002210A2250E202ACE2208C
:201CBC00214622F061FC61200421082295E125F0B5FF0446681D26F057F8242C40F094815A
:201CDC0000200BE2E878032800F2A481281D26F04BF80246E878DFF8AC1431F81010DFF83C
:201CFC00A804007825F0AFFF95E1E878032800F29681DFF8901431F81010DFF88C04007834
:201D1C001BF00AFB8CE125F0D1FEADF8080002AB61200C210BE1002661200E2101228DF8D4
:201D3C00086002AB94E1DFF8546401208DF810003068002800F034810069002800F0308121
:201D5C0002A925F074FF042122F048FE002800F0FD81044626F00CF8002800F02481214699
:201D7C00054625F09FF93068BDF80C1022462B4606690298B0478DF81000284625F0F6FF00
:201D9C0011E1DFF8F8432068002800F010818069002800F00C8102A925F049FF2068BDF81F
:201DBC000C1082690298904702E1DFF8D093D9F80000002800F00281C069002800F0FE8047
:201DDC0002A925F034FF05469DF808000024012809D1BDF80A0030B9BDF80C0069380328B0
:201DFC0038BF01246400284625F0BEFFAF788046F72F28BF6FF0080725F049FE002800F02B
:201E1C00A7810546ACB9D9F80000BDF80C10AA1CFBB2C469029800924246A047044640B9AE
:201E3C0000246120332132462B466F702C701FF03DF8284625F09AFF002C40F0C08080E1CC
:201E5C00681D25F091FF8146E81D25F08DFF8046092002AF242E18BF2F1808BF3526304627
:201E7C0009EB080525F0AAFE854201D9022060E1B9F1000F04D1304641463A4620F0A4FDC8
:201E9C00304641463A4625F05DFD002800F0F0800A204EE1E878012802D0002840F05181D4
:201EBC0025F0ACFA40F259600121ADF8080002AB61203CE00120EC1C8DF80800E220214628
:201EDC001EF0F8FC30B901200821224625F03AFD8DF8080002AB612003212FE1E878291D68
:201EFC00012800F0E980002840F0ED80E020E7E025F094FE0446681D25F036FF242C0FBFDA
:201F1C0000200146204625F003FE8DF8080002AB6120122112E125F081FE24280CBF002016
:201F3C0025F04CFEADF8080002AB61201321022205E1E8788DF8080091488068D0F8302443
:201F5C0002A9E02090478DF8100004AB61201421F4E08A4C2068C0B3806AB0B302A925F037
:201F7C0066FE2068BDF80C10826A0298904701462CE0824C206890B3C06880B325F04EFE83
:201F9C002168C96888472BE080466938002680B2032838BF0126681D082C45D1057846E017
:201FBC0003208DF8100004AB61203021C6E003208DF8100004AB61203121BFE00324002600
:201FDC008DF80840612033213EE0002104AC204625F03CFE6120322104222346AFE003208A
:201FFC0025F041FD3621A9E005F10806ED790146A8426FD92046002225F09EFC09288DF8C2
:20201C0008006DD1002D6BD020462946324625F099FC65E0022025F026FD0A218EE00220A5
:20203C0025F021FD0B2189E025F09EFE0546404625F0C4FD0227A84288BF7700FFB10026BD
:20205C008DF80870612021468DF8096002AB02221EF02CFF76E002988DF810400422ADF8F7
:20207C00120002208DF8110004AB6120082166E0012E60D1E22039461EF01CFC59E0471B39
:20209C00B8B2F72828BFF72725F001FD002861D01FFA87FB00F1020982464846594625F089
:2020BC0001F8404629465A464B4624F0CDFF0546002851D00A275AE00878022814D2522004
:2020DC001EF0F8FB00E002208DF8080002AB61200F2133E02046324625F02EFC8DF8080039
:2020FC0002AB6120072129E002A9522022F03CFAECE702359DF8080015F8016B012810D1D6
:20211C00BDF80A0068B9BDF80C8031462A46404620F05AFCB8F1010F03D1E22029461EF0A3
:20213C00C9FB3868BDF80C1032462B46476A0298B8478DF8100004AB6120214601221EF0BE
:20215C00B5FE0026304605B0BDE8F08F052028E7102434E7102772E78AF80170002761208D
:20217C002146324653468AF800701EF09FFE504625F0FCFD002D7FF462AFE2E7400E0020A2
:20219C000C01002060970200B8E80020FC9602002DE9F04F8DB08B46480714D45FEA0B407B
:2021BC0045D45FEACB4000F195815FEA0B6000F1BD815FEA8B7000F1D0815FEA0B5000F191
:2021DC00EE810020AFE1DFF814050178062900F2A881DFE811F007008F01A601A6019401CF
:2021FC00A6019B01DFF80055DFF8F4142A7891F82B30022A02D19E0600F193815E0700F1F1
:20221C0098819B0740F18D810423037091F82C30DB0700F0868191F82E30002B00F04B8281
:20223C0023F064FF0420012102F046FA50E2DFF8BC04DFF8B054DFF8A494DFF8B874DFF807
:20225C00A044DFF8B4A448F202080088019028781BF090F8002800F03A8106460078D3282D
:20227C002DD1F089404540F019813878002800F0158199F80000012840F0108124F0BEFFD2
:20229C00002840F00B817088002840F00781A24602AC1221204624F005FF25F0A3FB3046F6
:2022BC00214617F053FBBDF81400B0F5285FC0F08C80012002211DF0EBFE54462CE099F824
:2022DC000010884219D1012836D0032840F0E680DFF8140400780138012800F2DF80B078EC
:2022FC00012853D0002840F0D9807078002800F0BE8000201DF07AF8D0E00A280FD194F89A
:20231C002B00BA46B71C3071A16909B138468847384623F0E3FB5746DFF8DCA3BEE00928C0
:20233C0040F0BC80DFF8C0030078002840F0B680A168B01C8847B1E0DFF8AC030078013809
:20235C00012800F2AB80707860B194F8330094F83410013084F83300C0B2884202D901207B
:20237C00002199E099F80100032857D002286ED0012840F093803878002800F0888024F00B
:20239C003DFF002800F08E80012081E07078002872D025F0BDF94FF6FE71884203D1BAF81C
:2023BC001600884207D0AAF81610ADF82010532008A91EF07FFA1DF0BBF923F0EFFB002024
:2023DC008AF826001CF022F968E0CC48006807A908AA16F0F3F8074601985446DFF818A3E9
:2023FC00874212D29DF8300010B1FD208DF8300004203946142208AB22F058FAC04907EBD1
:20241C00470001EB8000012141720020012184F83200012002F050F9B64F3FE0A24608AC0C
:20243C00AB20002122461BF057FA042002945446DFF8C4A28DF80C0002A80EF001FE25F0F2
:20245C00D1FA28784FF4805141F288321CE0012020714FF48060ADF8200008A817F09EFF0A
:20247C0025F0C0FAA2484FF4805102680BE00FF011FC606990B9A5E702204FF4805140F608
:20249C00B83289F80200287825F0DDFB06E0002084F832000120012102F00EF9304623F0AD
:2024BC0007FED4E694F8350020B1E0690028F5D08047F3E70020002102220023ADF820008B
:2024DC0002208DF8280008A823F054FFB7E78BF4004028E0844800780138012859D87F48F8
:2024FC00017803294DD0012953D1417800201DF0CFFD4EE0012001211DF0CAFD11E023F0B5
:20251C00F5FD0420012102F0D7F80AE0002132220170734880F82A1072480421007825F0FD
:20253C0092FB8BF004000DB0BDE8F08F8BF08000F9E70522027091F82C2092072CD591F826
:20255C002E204ABB052202600120487000201BF081F8022023F064F8E3E76348007801384F
:20257C0001280BD80020CDE9080008A812F050FA20B15C48022100781AF02AFF8BF0020099
:20259C00D1E78178022904D10121817000201DF05BFD8BF48050C6E705200021B3E7524860
:2025BC000078002840F08480DFF834A1DAF80C50002D77D002A80130019008AC261D002D4D
:2025DC006DD0A87A18B10138A872000646D19AF83180B8F1000F11D00020A91C08228DF8D7
:2025FC002000304624F0A2FE204618F0E5FA28B12A88BDF82200314621F05EFFAF1C0DF118
:20261C001F012246384615F0D9FF8146384607A921F0B3FCB8F1000F05D09DF8300040F084
:20263C00020002281CD1DAF80800A0B101983946082224F07BFE022000220C238DF808006B
:20265C00BDF81C00ADF812002648007802A9009109211FF0A6F828461CF0A2FEED68AEE7D9
:20267C00384622F0FAF99DF81F000128DBD12046142124F017FD224A09EB4900002123463C
:20269C0042F8201002EB8000142241604172FF2049468DF83000042022F008F9C3E7DAF8A7
:2026BC000C0028B90F484FF4006100781AF034FE8BF4006037E7013A012A09D80322026097
:2026DC000120487001201AF0C5FF012022F0A8FF287800287FF425AF04205EE734E8002088
:2026FC0038080020C1E80020A80C0020AA970200480E0020980E002048DD00200CE80020E9
:20271C0050A300202DE9F04F89B020F099F8DFF8EC148122DFF8F084DFF8F0A4DFF8FC74E4
:20273C00DFF8F0E40A70DFF8D8140860DFF8D404FF2101700020DFF8E014A8F800008AF8E0
:20275C000000DFF8CC040968007891F808B04FF6FE718EF8000059448AB2B968D1F800315E
:20277C00DB899A421BD80422DFF8B844A8F80020DFF8AC24126893681D0ACEF80C30C3F356
:20279C000159AEF804501D0E2570D1F8B850B9F1020F2E780CBF002EB9F1030F10D124F02D
:2027BC0019F925F0BBFADFF8781400240A6813681C7112680A6025F0B9FA09B0BDE8F08F97
:2027DC00C3F30F2505F007050EB1002DE7D0DFF858C4042D9CF800C008BFBCF1000FDED0A6
:2027FC0036B1DFF848643678862E01D1022DD6D19D0216D403F4E063B3F5007F08BFBCF1EB
:20281C00000F1ED0DFF824140978862909D10020754620F04DF8DFF81004AE4690F800C02F
:20283C002878BCF1000F49D1002847D00128B6D003283CD0022841D1BEF804004007AED125
:20285C003CE0D1F8D40090F88300022877D0A1460520147BF246A8F8000025F05FFA0546FB
:20287C00DFF8C8030078862866D1B868016C096811B9D0F84C05804760B20021002625F027
:20289C00BDFAB9680A6C12685077086C00688677086C0068C477284625F048FABAF8041012
:2028BC0099F8000001F010011BF004FF47E0BEF8040000F0070003287FF471AFBEF804000B
:2028DC0001073FF56CAF810402D481053FF567AF9EF80E10C1F38105012D3FF460AF8E0965
:2028FC00012E3FF45CAFB9F1010F11D840F0020101F0070103290BD155EA06013FF44FAF01
:20291C0035B9B968D1F8AC10097800293FF447AF4FF6FB71B9F1020F594413D1C54A535D88
:20293C00925D02EB030945EA0602430615D4002A18BF09F1020914E0284625F0F7F923F0AA
:20295C00F9FD2EE7BA4A535D925D02EB030946B1420648BFA9F1020903E0002A08BF4FF0B6
:20297C000209C0F300205FFA89FB8BB2ABEB00028EF801009A423FF712AF0844B968A0EB59
:20299C000B00AEF806007430D1F8501280B28847A049002888603FF402AF7421CDE901B9B2
:2029BC000396AB4624F07EFB9A4F0020B8709E48007820B9387900F020008AF80000787849
:2029DC009AF80010964E4FF000092546002993492CD000284FF0000029D1B88800F0070009
:2029FC00032807D0012821D18868D0F8D40090F88200D8B1C8684069007818B124F0B2F9A6
:202A1C00FE280DD085488068D0F84C02804738B982488068D0F844028047002800F0EA800B
:202A3C007C4F0120B8707E4E254600E00020BC6804F1740184F83AB06160A1657978BB8840
:202A5C00FA880029A381039B228184F830302B7808BF994697F80EB084F84990A4F85C206B
:202A7C00FF22B8F80030A273CBF301195D1A797B029FA8F8005001F0780160F3820101EB24
:202A9C0009002074380600F0AD80306804AE019A10FA85F000F10801304625F0F5F955FAFC
:202ABC0087F0CBF38105A8F80000207C00F04007E5B3B9F1020F00D13FB9BDF810000236B3
:202ADC00A4F84400A4F8420002E0B4F8440004AEDFF86481B8F80E10884204D04FF6FF71BB
:202AFC00884240F08280032D12D104F13200314625F0FAF8474C08F10301A068323022F0FA
:202B1C0059FF4649002870D094F80EB008360FE036F8020BB8F80C108842608606D04FF601
:202B3C00FF713C4C88423D495FD101E03B49394C0020B0EB9B1F22D04FEA9B10B9F1020F11
:202B5C0008D157EA05010DD136F8021BA268A2F8421007E0A1680A7C52065CBF36F8022BD6
:202B7C00A1F84220032806D1A0683146283025F0BBF8284C02E03088A16808852749A08861
:202B9C008968B9F1010F11D8D1F8AC2012786AB140F0020202F00702032A23D135B9264A9D
:202BBC00A368D289B3F8423093421ED100F00700032806D0012815D1D1F8D40090F8820004
:202BDC0080B1A068D1F848128847124E50B90020F17BB070B07BC1F3011100F078000844F4
:202BFC00B168087408F01CFCDBE516F080FC18F04BFAD6E5074FB87815E700BFCEE80020B3
:202C1C0060E80020D3E80020CEE40020D1E80020D0E80020AC0B0020A0E800200C01002026
:202C3C00F8E70020E1E80020E0E80020D6E800204C9702004897020020E700202DE9F04F88
:202C5C009BB0DFF808650546DFF8047530780328387040F04D81002000211822082330706F
:202C7C0038700CAC204623F0FDFE2046002121F049FEDFF8E0B4B8603A21584624F012FAE9
:202C9C004FF0FF30ABF81400CBF81000CBF80C0021F078FB002029461CF04EFF07F11001DC
:202CBC00F86024F0B2FFD7E90502DFF8AC54B0FBF2F1C9B2032928BF03218BF800102970D1
:202CDC00B2F5005F40F01281B0EB413FC0F00E81F868002800F00A814FF40050DFF880A424
:202CFC004FF00008FF22ABF80600FF208BF803208BF8058004900020079000200A900020B5
:202D1C00089000200690002005900020099000200B90FF200190FF200390FF200290CCB28F
:202D3C00A04580F0E8805FFA88F600211AAA0423304624F0CBFA3046002119AAD0473046A1
:202D5C00012118AAD0473046022117AAD0471A996FF06F0050FA81F2C8B20E2A06D80123F9
:202D7C0003FA02F245F201131A4203D1A0F1FE02022A04D242F28352B2EB914F1AD0304652
:202D9C0013F018FD0028387040F0F080304600211AAA042324F09AFA3046002119AAD047F4
:202DBC003046012118AAD0473046022117AAD0471A99C8B208EB48020BEB8209C1F3014233
:202DDC00090A4C46FE2804F8160F61709DF86610E270A17001D3102105E0BDF864104FF654
:202DFC00FF72914223D0A9F81C109DF86210702889F81A10BDF86010A9F81E109DF85E1072
:202E1C0089F81B10BDF85C10A9F820102CD078282ED07C2830D07E2834D0FE2839D0FF28BA
:202E3C003DD10798CDF80880013007903AE012A81FF09EFA304600214FF088524FF40053F3
:202E5C004FF0885B4FF4005724F040FA4FF6FC724FF0885357B3043F07EA020000F1885B6B
:202E7C00C058411CF6D024E009980130099019E005980130059015E00698CDF80C8001301B
:202E9C0006900FE00898013008901FFA88F0019008E00A98CDF8108001300A9002E00B98D7
:202EBC0001300B90297808F1010838E7DBF80000002701210126CAB2042A06D8C2B2FF2A00
:202EDC0018BF0E460131000AF5E7CBF80000A548129900684268A448904757FA86F09C4FB1
:202EFC00DFF870B2A9F81C0020787EE7012030701BB0BDE8F08F0B9800060BD10A98C0B2BA
:202F1C00012807D80998C0B2012803D80898C0B201280FD99148042200240270CAB2E0B2B0
:202F3C0090420ED213F046FC39780134084329783870F3E7079BD8B2A04219D18748002241
:202F5C00027000208BF803008BF80100481E7E218BF80200BBF81C00ABF8060000201FF088
:202F7C00D9FE9BF80200FE211FF0D4FE3878BFE70998000624D00A98049A000603D1029A22
:202F9C00180600F08380754802210126D5B28BF80220017016FA82F0B0FBF4F101FB14003E
:202FBC008BF80100284613F005FC38702846FE211FF0B0FE8BF80560002000F0D7F8D5E78A
:202FDC000A98049A000621D0644801218BF80220017011FA82F0039AB0FBF4F101FB140000
:202FFC0091B2FF298BF801001FD10199FF2919BF8BF8031001EB41008BF8030000EB4000C8
:20301C000BEB8000808BABF80600AFE7DDE90520104300063FF47EAF21F088F9A04280F04C
:20303C0084804E48032101703DE048008BF8032010FA82F00BEB8000818B1829ABF8061042
:20305C0094D30739D0B212AA89B215F07DFB9DF853004007B0D53F49BDF85620002300939A
:20307C000323C878C988891A12AA073989B206F081FF00287FF47AAFBDF8541000293FF4F4
:20309C0075AF9DF858001BF0C3FF6FE721F04EF90621A042314838BF03210329017002D07C
:2030BC00062952D062E721F041F904468BF80C0000EB40000BEB8000408BABF80D000CF01E
:2030DC0011FB29782044B0FBF1F202FB11008BF802000130C2B2B2FBF1F202FB11008BF8DC
:2030FC0001007C201FF030FEFF2812D17E201FF02BFEFF280DD1FF201FF026FEFF2808D1A3
:20311C0078201FF021FE01469BF80100FF2918BF0846C1B28BF80300490051FA80F00BEBB2
:20313C008000808BABF806001BE70798000609D0DFF820B0FE219BF802001FF0EBFD2C78C9
:20315C00029A41E7054806210170FEE7750E0020D800002090E10020B9E80020C5E800200B
:20317C00E1740200D8010010004003402DE9F04F9DB00446DFF8D804406818B18047002871
:20319C0000F04A82DFF8CCB4DFF8CC240A940DF1380A4FF0F8089BF80000411E002C0B9162
:2031BC0018BF0121D17392F8029002F118045178002700250D91C0B287421ED2B94517D0C8
:2031DC00FEB2002152460423304624F07FF80E9810F4403F40F0040018BF0135C0B27C28C2
:2031FC0006D130460621F82223F000F884F800809BF800000C340137DDE7E9B20138002259
:20321C00DFF85474884203D17879002800F01C82DDF828A00DF154085046BAF1000F08BFA0
:20323C0010200590002001900D9E0B9D0024280400F0CE81F87B08B90120F873F0B2002197
:20325C000EAA042324F042F80E98BAF1000F15D010F4403F15D04FF400509BF8001001340D
:20327C00013D3882F87B0138F873012050FA86F0B0FBF1F202FB11067E73D8E7002102913C
:20329C0002E00D960B9502940026C0B2702804D00D987021C0B21FF03DFD5FFA89F400216B
:2032BC000EAA0423204624F011F89DF83800FE2803D02046FE211FF02DFD20460621FE225F
:2032DC0022F094FF4FF400500D9D07F11601BE82DF4E002287F80C900C943882FF20B87393
:2032FC00E8B232707D73400050FA85F001EB8000B0F806A060009BF8004050FA89F001EBEB
:20331C008002FE20A7F812A0FF7B114601F8020F32F8060F04910990039214A81FF028F8D8
:20333C0057FA85F0013890FBF4F101FB14000090099807900020CDF818A0089000200D992F
:20335C00CDB20C998D4200F09880C00740F098801FFA8AF0162871D93078002840F0568155
:20337C005F46AAF1070B28460FAA1FFA8BF4214615F0EAF99DF8460096281CD1BDF84A60EC
:20339C0006F11000A04216D89DF84700C10701D1800703D40020ABEB060A2CE0ABEB0600F8
:2033BC009DF8452031462B4684B2204618F074FA20B3AAF1080B1FFA8BF01728C0F0268152
:2033DC00ABF1160436282846424688BF2024ABEB040BA3B21FFA8BF123F078FF2004EAD045
:2033FC0018FA84F010F8010C962801D0013CF5E704EB0B0A0020964EBB46A0E7F01D83B29C
:20341C00079813FA80F1B1F5005F01D90120F2E780B28A46934918440A1A2846214623F054
:20343C0055FF089801300890BAF5005F07BF01204FF40051514600200791ACE7089810B1E7
:20345C00854924F085F80098C0B2854200F0BD800D99012050FA81F09BF80010B0FBF1F240
:20347C0002FB11007C490D9000EB400001EB8000B0F81CA0079809905CE70C9D01240BE091
:20349C00089810B1744924F063F8DDF8349000240798CDF818A009903078DDF828A00028A4
:2034BC0040F0B48009981021C0F50052103883B20C98C1F200121EF077FF317808431499A8
:2034DC00307066480068426865489047624F06987CB19BF800002918013991FBF0F202FBF7
:2034FC0010195FFA89F0400050FA89F007EB8000808BB882099903980C9CB7F91220012310
:20351C0087F80E9001803982797B204620F024FFB7F91420B97B2046022320F01DFF388A18
:20353C00029CBAF1000FC0F5005004D005998842A4BF01210191059988424FF07C01B8BF24
:20355C0078210C9E30461FF0E5FB0CF0CBF80546F87B0621FC22401BF873304622F046FE53
:20357C000499FC20BB7B0870B97815FA84F00D9301449BF80000B1FBF0F202FB101909F1EE
:20359C00010187F80290CAB2B2FBF0F202FB1011797003EB430107EB8101898B102906D120
:2035BC000D990131B1FBF0F202FB10100D900B98401BBAF1000F0B903FF436AE019880F05C
:2035DC000100C0077FF430AE02E0DDF800905EE77C201FF0B9FB0446FF2823D17E201FF0B9
:2035FC00B3FB0446FF281DD17C7804EB440007EB8000807DFF2811D09BF80000B9780144FB
:20361C00013991FBF0F202FB10140BE0134814990068426812489047002215E020467E2173
:20363C001FF078FBE0B2FE21FC70400050FA84F007EB8000808BF880B8781FF06BFB002017
:20365C007871388AC0F5005210B21DB0BDE8F08FD8000020B9E8002090E10020D8010010B6
:20367C0000400340002000112DE9F84305460C46480414D4A00023D4A0075DD4600500F193
:20369C008080200500F10781200700F13C81600040F1F78018F004FD24F08044F1E024F0CD
:2036BC003DFBDFF824140F6D3FB1D7E90A1202F0E04201F00A01891848D024F037FB5DE013
:2036DC00BC48DFF80874016841F080010160B878012804D104201FF085FB0020B87024F0BE
:2036FC001DFB0646B448406D016804208847DFF8E4130A68904219D12A7EBAB1FA68AAB179
:20371C00DFF8C403806C002800F09880C16840F603020988914206D0C06840F6040100884A
:20373C00884240F08B8005F1140089E040F6C4120860C5E9042285E009F036FADFF88803BD
:20375C00006C002808BF24F002049AE0D7E90A65D7E90A12AA43B143C7E90A1224F0E6FAB2
:20377C0056EA0501B86818BF002807D0D7F808C03869B7F9301032462B46E04724F48044DD
:20379C007FE024F0CBFA054621F0A8FE002800F0B780CD48876B002F00F0B280DFF82C83A6
:2037BC000420CD49002288F81800C74822F069F824F043FAC94824F0ABFAC5480068006B7C
:2037DC008047C8F810000125042088F8025020F045F8386990F82810C8F80400490703D580
:2037FC00436A04210022984701201AF0A9F9D8F80400457611F070FBD8F8040081680B4604
:20381C001A465B684BB11E88A6F60306072EF7D805FA06F616F0830FF2D0537B03F0F00315
:20383C00013353730023FD6853602D88A5F60305012D00F28A80C8F810309FE005F1100030
:20385C001CF006FF304624F071FA20F01FF878B12E6A28466FF4807100224FF00073B047D1
:20387C009948806B10B118F01BFC01E044F00204EE692846002100224FF08063B04724F030
:20389C00005434B1984821462830BDE8F84324F085BABDE8F8838D4EB078012804D10420BC
:2038BC001FF0A0FA0020B0701FF0F0FF38B170686FF4807100224FF00073056AA847306925
:2038DC0050B183480068006B804732697168801A000BC860002030617B4D82490022284651
:2038FC0021F0CFFF02203076286C20B17E480221283024F053FA18F0D3FB24F40064C0E705
:20391C0024F09BF941E024F009FA054621F0E6FDA0B1DFF8B88198F8000000070ED498F901
:20393C00000000280AD4684612F05EFA08B1009820B1DFF8B89199F8610048B324F07DF9A4
:20395C0018F0AEFB24F008049BE7034633F8385FA5B190F8445090F8456005F0F00580F8EC
:20397C00445006F0F005013580F8455000255360C5634587507B00F0F0005073584800226D
:20399C00C2610160012022F009FA24F4806478E700260127602E11D009EB0600817A31B162
:2039BC008772407A07FA00F0C0B21FF035FA2036F0E700BFCC2108408C010010032088F836
:2039DC001800464824F0A4F924F037F9444F3E4D0022786900207861F968F8602846444962
:2039FC0021F04FFF3A480068006B8047D8F80C10D8F82020411A02EB1130B0EB113F38BFC9
:203A1C004FF0FF3098F82410C8F8200021B1D8F80810B0EBC12F20D922F0D0F9B8B140F6C0
:203A3C000900414621F83C0F002048804A7B02F0F00201324A730A7B02F0F0020A73486067
:203A5C00F8613960B8F83E0010F4406FFAD00020C8F82000012088F824001CF001F82548B6
:203A7C00002101600220002122F098F902201FF0B9F9102010F0B6FD98F8010020B9D8F8C2
:203A9C000400503024F082F91B48807810B90D2010F0A8FD98F8250028B1002088F82500AE
:203ABC0005201FF09FF9002088F818001348C8F81C000220B5F85610B5F85420914208BF3F
:203ADC00072017F005FD3BE7B8060020900500208C010010B40D0020D554020010E000202C
:203AFC000010044025000100F8050020C0DD002021C1010000000460B496020011F90000B9
:203B1C002DE9F04F8DB084780226142C00F216820546DFE814F02900150015004A008800CE
:203B3C001302130213021302130213021302130213021302130291009F00B200C100CF0010
:203B5C00012095F80180022C8DF8310040F0C380E878291D03288DF82C0040F0E38009A8FD
:203B7C00082223F0E3FBE2E010208DF82400102024F0FEF898B10446DFF8CC0321466060D9
:203B9C00E81C0FF08DFB8DF8240028B9204621F023FD8DF8240010B1204624F0E7F8002674
:203BBC0009AB642000210122B9E101208DF832000020CDF82A00ADF82E00CDF8260002200C
:203BDC008DF82C00E81C24F0CFF8ADF824006979A8798DF82D1023F039FC8346E81D24F081
:203BFC00C3F895F80C908046687AAC7A95F80BA04FEA49078DF83100384624F0B9F8002815
:203C1C0000F00681CDE9074806464FF0000805EB080047456FD00D3024F0A6F826F80800A1
:203C3C0008F10208F3E7E8781FF0C6F98DF8240009AB642004217DE1E978032900F24681B3
:203C5C00281DDFE811F0040045014901510117F0E1FC6AE1E81C24F087F8BA4C6668002E8D
:203C7C0000F0DA806A79002A00F0DA803368A91D184423F05BFB0020CFE0B24EEC1C042165
:203C9C002046376820F0AAFE002F49D0B968814200F096803F68F7E7A888ADF82400E8783B
:203CBC0009A922F091FB8DF832000DF13203642013213FE10026E878ADF8246009A921F064
:203CDC0035FEBDF824000DF1320314210222ADF83200642023E1E81C02218DF82C1024F0D5
:203CFC0043F8ADF824000020AE1DADF82E0068798DF82D0026E0BBF1000F00F0AC80437BB8
:203D1C000DF131010E30CDE90496CDE9000107985946CDE9020A09A8089A1CF066FB9BE0D7
:203D3C000120F5E0084624F01FF8ADF82400287B8DF82D0005F10D0024F016F8ADF82E00E2
:203D5C0005F10F06307823F081FB0546701C24F00BF88146F07896F804A096F805B0022C45
:203D7C008DF8320008D1B01D23F0FEFF074606F1080007F10A0102E0B779F01D39463DB1DF
:203D9C000A3189B2FB2905D36E4E706800286DD0022009E00DF132018DE8030C09A84A469B
:203DBC003B46294603F0B0F88DF8310008F0E000202840F0C2800DF1310364202146B9E05E
:203DDC00EC1D204623F0D0FF6D7A002D00F0958005F102098246484623F0CAFF002800F012
:203DFC0096800026457080462A460670786800EB0A0108F1020023F099FA5FFA89F264203B
:203E1C00122143461DF052F8404623F0AFFF95E010208DF8320024E010208DF8240016E0FD
:203E3C00D6F800C0F38AB28A3169757EB77E06F11800CDE900C0301DCDE9025703F064F82D
:203E5C008DF82400606823F091FF0020606009AB642011216EE002208DF83200304623F038
:203E7C0085FF0DF132036420032163E007F11C0023F07EFF0028706054D000F11C010C2288
:203E9C00016000208DF83100706809A9043023F04DFA70680F214FF47A720561C1769DF84E
:203EBC003210294DC782A0F8149080F81AB080F819A001762878082123F0C5FE00283FF4C5
:203EDC0075AF2878082119F083FA6FE702202CE0007818F0B1FD28E0007823F0B7FA18B392
:203EFC0022F0A4FF002020E023F03EFFA97923F0ABFCB0FA80F0400917E03068B84201D1E7
:203F1C0038683060384623F031FF002000E0102000262070642012210222234666701CF088
:203F3C00C5FF0BE010203FE701208DF8240009AB6420102101221CF0B9FF002630460DB0ED
:203F5C00BDE8F08FEC0C0020B8E800202DE9F04F8FB00C4608040BD4A00425D4DFF87C5335
:203F7C00287802282CD1E1077CD1A10641D558E0DFF86003007819F0FDF990B10178DFF8F2
:203F9C00582305460020602808D0135C08308B42F9D1104450F8041C28468847284622F008
:203FBC0087F884F4004591E11CF002F928B10546FCF744FE284622F07BF884F4005585E1B1
:203FDC00A1062ED4012814D8E10600F11381610600F12B81210600F13981E10500F13B8132
:203FFC00210500F13D81E10400F15081610400F15781A10700F1DE80A10500F1F6802107CF
:20401C0000F10D81610500F11581E0034FF0000540F15C811AF0EAFCB348C57084F4803596
:20403C0054E1AC4F202138781DF000F8DFF8B882D8F80810084324D023F062FE054623F035
:20405C002BFBD8F8081059B168434FF47A72B0FBF2F0401A4FEA500538BF6FF000458DB9FC
:20407C00002570E0A44890F82C100F2906D190F82600022802D300201EF0CEF984F00105D4
:20409C0024E1012500200421002220F0A9FF06464FF006094FF0FF084FF6FF7A0DF1080B0B
:2040BC00002E4DD0304604210022374620F098FF06463889401B38BF002038810004EFD1BC
:2040DC00B87BD0B301280AD17889400707D4386887F80D90B721407B1CF022F8E0E739680A
:2040FC005A468DF80680ADF804A0086AC97F0CF003F901281BD1B87BB97A8DF838000907B6
:20411C00788A40F08002ADF8362006D540F4C070ADF83600387B8DF83A00786910B1007B2B
:20413C00ADF81800584601A9002202F0A1F9387B87F80D9015F05CF8B2E701207873AFE74D
:20415C00DFF8A481634F21F06FF800200121002220F046FF18B13878202119F039F900204F
:20417C0004210022002620F03BFFC8B306890421002220F035FF28B10289B1B2914228BF56
:20419C001646F4E7A8B2B1B2814224D988BF08462021401B80B24200387823F054FD23F083
:2041BC00AFFD054623F078FA68434FF47A71B0FBF1F615E05148007808B302AD284623F00B
:2041DC00B5FC23F093FA4E490B784E490A78294619F032FC20E03878202119F0F9F8002688
:2041FC00C8F8086084F0200570E014F0BDFC84F400756BE007F07AFC84F0100566E03E48DB
:20421C00418B012023F0AAFD2878022804D131480121007819F080F884F0020556E032487D
:20423C00012184F00805817050E00BF0E7FB84F040054BE0022808BF14F0DAFE2E48012178
:20425C00808C23F07DFD84F480653FE022F07EFA84F080053AE020F01FFD84F4807535E0E2
:20427C001AF02CF91E48007801280CD11D48007848B14FF47A7100FB01F216484FF400611B
:20429C00007823F0DDFC84F400651FE01648017819B1002101701AF011F984F4805515E039
:2042BC001348006880B11149097801290CD180471048006800B1804706484FF480414FF478
:2042DC007A72007823F0BCFC84F4804528460FB0BDE8F08FBAE800204C900200A80C002091
:2042FC00AB0E0020AA0E0020600C0020A80E0020DC090020E809002048DD0020840E002082
:20431C00AE0E0020B00E00202DE9FE4F8846080426D45FEAC87004BF0020BDE8FE8FE548CD
:20433C00056823F0EDFC044623F0B6F960434FF47A714FF6FF72B0FBF1F14FF6FF70002DF7
:20435C0000F01A812B886C88CB1A9BB29C4240F21C81E31A94B2A342B8BF1A46ED68EEE707
:20437C00DFF840A3CDF804809AF8000019F002F8002800F0FC8006460078012840F0EC806C
:20439C00DAF8041096F83390D6F814B096F8138021B148468847002840F0DE80718896F8AB
:2043BC003100022220F0D8FB0546002842D0287A297CA0F10108FF2900F0BB80707F4F466C
:2043DC00C00718BF0027E97C287D0144B94204D8E974FF2101FA00F06874A969A87C96F8CE
:2043FC003020896A10FB0710F16A22F09FFF287D697CB7FBF0F202FB107001228240D2B22D
:20441C000A436A74C8457CD196F83010AB7C13FB0713A9698B844FF4FF7303FA00F0C0B2A9
:20443C001043FF2868746CD1287C19F05DFBFF2028747FE0707FC00700F08E80B07F23F0B8
:20445C0005F8002800F0888004461C2023F090FC002800F081801C21054622F023FEB07FFB
:20447C0002A921F063FA9DF8090002212875284621F0E4FA708896F8312096F8301096F819
:20449C003330A880287DEA71FF2202FA00F0687460680078A9742874302013FB010080B202
:2044BC0020F08CFF0028A8615DD004461A20B11C2060708CA080A01D21F094FFF27F04F133
:2044DC003000B17F96F82830C4F81CB084F81980A062307CE273744A217563750121A07577
:2044FC00928C2282F28EA285F28C6282B6F81100A4F817009AF8000085F8089018F068FF4D
:20451C0055E723F0FDFB044623F0C6F860434FF47A71B0FBF1F065492880634809780079C5
:20453C004843642148436249097800FB0100688000E04F46E87C297D6A7C01440139B942D5
:20455C0018BFC8450CD186F83300708806F11C0186F8342015F080FD304621F0A9FD03E756
:20457C00FF2AF9D1EFE7284621F078FAF4E7019880F40040BDE8FE8F92B282424BD0494857
:20459C000121007823F05FFB45E0A879022806D1287CFF2837D0A86921F08AFD33E023F010
:2045BC00AFFB044623F078F860434FF47A71B0FBF1F03F49288095F83800097888421BD2DE
:2045DC0095F83620FF2A06D195F83720013085F8380085F8362095F8351095F8394082F0F5
:2045FC00FF0300200126C7B2A7421DD206FA07F71F4214D10130F6E7EA8BA87E95F82A1051
:20461C00E9231DF045FB284621F028FA25480121007818F0DDFE88F00100BDE8FE8FFBB242
:20463C0001441A4385F83620AB8F95F83440C8B204FB10339EB2A64203D2FF2285F83620F1
:20465C0002E0FF2A08D12346184A174E1278367972436426724302E095F83A2023466A80E1
:20467C002A8D0E0606D022F0200244432A852A6C224404E042F020012A6C2985297A85F87C
:20469C002E10E9796A6285F82D10D9B269840549496811B188470028B8D105F1100004F025
:2046BC00ADF8B3E7CC0C002048DD00209E0E0020A40E0020CCC200207FB50138072800F288
:2046DC004A810C46DFE810F008002A0052006C0087004701A400C700CA48007801380128C4
:2046FC0000F23981002C00F045810020032100241DF0AEFCC54DC64E042004213222287096
:20471C00307823F0A0FA0820002106F051FA30784FF480516C7018F0FFFD7FBD0020002581
:20473C0022F09CFEBB480121017004208DF80D0074B1B548B34C45852078012803D10720BE
:20475C0021F07CFB2078022802D1062021F076FBAE48042132220570AD48007823F073FAA7
:20477C00A94890F82B1001F0FE01F2E0A54800780138012800F2EF80A548042132220078A1
:20479C0023F061FA002C00F00F819F4C9F48012101702069002800F0EC801DF0A9FFF8E7DD
:2047BC000120002C8DF80D007BD0974800219B4A80F82A10984823F005F8924C207801288D
:2047DC0003D1072021F03AFB2078022870D1062021F034FB6CE002208DF80D008A48002C15
:2047FC0073D000218D4A80F82A108B4822F0EAFF002003211DF02CFC824C2078012803D106
:20481C00072021F01BFB2078002877D1092073E07C4D00208DF80D00002C28787BD018B947
:20483C00092021F00BFB2878022806D10820002106F0BEF9042021F001FB13F021F973487C
:20485C000021C822017070480D2180F82A10704823F088F978E005208DF80D0069480078A4
:20487C00022878D1002C00F0C38068480022C178C270017042F20800002106F099F962480D
:20489C000D2190F82B2080F82A10C17802F0DF02002980F82B200CBF04200D2021F0CEFA5C
:2048BC0059E05848007818B95748022180F82A105648002132220170554823F053F952482C
:2048DC0090F82B1001F0FD0143E0082180F82A104C490978012911D890F82E0070B90020E4
:2048FC000DF10A018DF80A0052201BF0E3FF22F029FB1DF047F8002021F0A0FA43480021AC
:20491C0032220170424823F02DF93F4890F82B1001F0FB011DE03C4C022812D194F82E0070
:20493C0078B194F82B00002140F0200084F82B0005208DF80D00082006F03AF90A2021F020
:20495C007DFA022084F82A002F4890F82B1001F0EF0180F82B102C480022032390F82A00C0
:20497C008DF80C002A48007803A900910A211CF018FF7FBD244C0720254D4FF4805184F840
:20499C002A0001208DF80D00287818F0C5FC0020002620F085FA2878022141F2883284F8B4
:2049BC002B6023F050F9D6E7174C022000218DF80B1084F82A001548017094F82B000DF1C8
:2049DC000B0100F0FD0084F82B0001208DF80D0052201BF06FFF22F0B5FA1CF0D3FF0020BE
:2049FC0021F02CFA20690028B5D01DF081FEF9E70548022180F82A1090F82B1041F020018B
:204A1C00A7E700BFA80C00203808002034E80020C1E800209B0E002048DD00206E0E00204A
:204A3C0092B0DFF8E892D9F8000010B1002180F8451048301FF0DAF823F070F98046072085
:204A5C0010F03EF816F07AFD10B1B14823F06AFB19F0CEF801AD284622F0E0FC0427002031
:204A7C0029468DF8047022F0E1FCAA4E306022F00BF90AAD284622F099FB002029468DF846
:204A9C00287022F09BFBA44C206022F007F906AD284622F09BFB002029468DF8187022F0C1
:204ABC009DFB21689D4D286019B99D4823F03AFB286810B99B4823F035FB306810B99A4886
:204ADC0023F030FB1BF078FAD9F800004FF0FF3658B1CDE9106610A9082221F095FB411EA2
:204AFC00D9F8002018BF114600E00021CDE9106621B18E48082222F019FC17E0082023F023
:204B1C0037F9D8B305460024052C04D822F0CEFF28530234F8E74FF6300029460822E8805D
:204B3C00824822F003FC284623F020F910AA0120082122F001FF092800D0D8B91FF0F6FF38
:204B5C00800712D4CDE91066CDE90E660EAB01200021082222F078FA60B90EA810A908221B
:204B7C0021F052FB002800F0CB80704A0120082122F0E8FE6D49E2201BF09CFE11F002FC00
:204B9C00282023F0F5F86A4E0028306055D0694F694C07F10C0522F0E1FF22F05FFB3068B0
:204BBC00056007F1100522F0D9FF64498968D1F84C1388473068456007F1140522F0CEFFBB
:204BDC001AF0DCFD3068856007F1180522F0C6FF18F060FA3068C56007F11C0522F0BEFF66
:204BFC001DF094FF3068056107F1200522F0B6FF1CF040FF3068456107F1240522F0AEFFAE
:204C1C001BF0D0FD3068856107F1280522F0A6FF21F020FE3068C56107F12C0522F09EFF81
:204C3C001EF06CFF3068056207F1300522F096FF387022F04BF93068456217F025FC40481F
:204C5C0040494FF00009CDF8409001603E480321119010A81EF0D2FD22F0B2FC404623F038
:204C7C0065F816F079FD22F044FF01201CF09EFB18F094FC36480078022808D133480078A0
:204C9C00012804D14FF40040012105F091FF294F4FF48041387822F0A7FD2E484FF0FF3109
:204CBC00006823F03BFADFF8B08078684FF0FF3123F034FA3068002550F82510096821B90C
:204CDC00691C092D0D46F7D3EFE722F01DFA316851F825100C68C1F8009022F07FF858F834
:204CFC002520002021469047044622F00DFA316851F825100A6822430A6022F06FF8D4E706
:204D1C000A480EA9082222F011FB33E7400E0020B49002001CE8002020E8002024E80020E0
:204D3C00D2900200E5900200F8900200D6E7002098E80020B4040020CD2D02000C01002074
:204D5C00F409002081B40100008D1500C30E0020A80C002074E80020CC9302002DE9F04F4B
:204D7C0089B08A4608040DD45FEACA7040F01C815FEA8A7000F12A815FEA0A7000F132818B
:204D9C00002041E1A24F387818F0F4FADFF88892A04C06464FF0000B48F21508002E00F036
:204DBC0000813078312837D0322848D0D32840F0B280F089404572D0382840F0AC80CDF8BE
:204DDC0020B0CDE906BB304606A91EF0EFFD9DF81C10052967D8307B002840F09C809DF86F
:204DFC001D000138042800F29680069821F0C7FE002840F09080707C88490DF1180C78706A
:204E1C00708808809DF81D00214601388DF81D009CE80D000DC17EE0B87803287BD899F806
:204E3C002E10814821F0ABFE002874D1FF207D49607170880880B088794908806BE060794C
:204E5C00FF2814D0002015F0F7F90246B9F8701078783346CDF800B011F044FD607900287C
:204E7C0059D038780821322222F0EDFE53E099F81810706820FA01F2D2071ABF3144097A48
:204E9C00002106F1080200231B2B42D020FA03F5ED0702D0D55CA9421ED80133F4E73046EA
:204EBC001FF05EFF37E0FF293DD0FE2956D199F872109DF81E00884202D860BBFF292AD128
:204EDC001BF01CFB069900201B2859D021FA00F2D20757D10130F7E7B9F86E004F4933461C
:204EFC0008804F4802884F48018810200090002011F0F8FC0120F870B87840B93C200221C7
:204F1C004EF66022B880387822F09DFEB8780130B87084F805B0304621F0CAF8387818F05F
:204F3C0029FA06463AE799F872109DF81E00884203D80028EFD1FF29EDD11BF0DFFA06980A
:204F5C0038B1D9F82810814203D0C9F8280020F085FFBDF8200021F0B9FCDCE7307B0028FF
:204F7C00D9D170882D49802200230880707CCDE900BBCDE902BBCDE904BB10F0AFFBCAE710
:204F9C001B2000E0C0B299F818108142C3D02749087099F80700642100FB01F23878012194
:204FBC0062E78AF400402FE020491B4C08782076E1201BF07FFC20F051FF0020A4F87000C6
:204FDC00012015F039F98AF001001DE010488188B1B101394EF6602281800078022122F074
:204FFC0032FE0FE00B4C607938B12179206821F0C6FD10B96079013860718AF0080003E056
:20501C00002181708AF0020009B0BDE8F08F00BF540B002078E7002048DD0020B2E700204E
:20503C00CAE10020CEDE002000F8FF07BDE800202DE9F04F85B08846080418D4AA48007840
:20505C00012802D85FEAC87155D15FEA88714CD4022807D1A5480078012803D15FEA4870C2
:20507C0000F188805FEA087057D400202DE1DFF860A29AF8000018F07DF9002800F023815C
:20509C000546807FC8B9688C132816D191486E8800F11C09002049464F46002818BF071DC7
:2050BC00086850B1014631F8042BB242F4D144683C6022F05BFE2046F3E7A87A05F1020BF3
:2050DC00022840F0E680DFF80C9295F83170BBF8006009F11C000068A0B10188B14202D120
:2050FC008178B94242D00430F5E77A480121017088F00200E9E07748406900B1804788F08E
:20511C000100E2E0D9F81C40002C57D001206168002955D001300C46F9E77148DFF8B491C0
:20513C00807BD9F81C60000760D422F0E9FD044622F0B2FA6B4A60434FF47A71B0FBF1F0BE
:20515C00D9F818101288411A91427CD3B1FBF2FB0BFB02F2511A08445F49C9F818001FFA3F
:20517C008BF00978884288BF8B4641E05A490978C170A5E05F495E4800224FF6FE730024F0
:20519C000978023079B130F8025C9D4208D04588013D45802D0406BF027020F8023C012426
:2051BC0001390630EEE734B1494804214FF4FA72007822F048FD88F0040086E0002400204F
:2051DC00464980B20988884263D2082022F0D0FD00285ED000210680877041603E490978BE
:2051FC00C170D9F81C1089B3606041E04FF0010B00205FFA8BF44FF0000A071D002808BFA9
:20521C0009F11C07A6B1F078A04298BF2046A0EB0B00F07006D8756830463D6022F0A6FD7E
:20523C002E46EFE7716830460AF1010A0E46E4E75FEA0A4007D100200821C9F8180024489B
:20525C00007818F069F888F008003EE0C9F81C002348807B00070BD422F052FD044622F0CD
:20527C001BFA60434FF47A71B0FBF1F0C9F818001B48807B00070CD59AF8000008211BF0BB
:20529C00D5FE30B91748082102889AF8000022F0D7FC2878022810D0012811D1297EAA891E
:2052BC00EB7C05F11C006C696E7E8DE85A0005F11003594604F094FD02E0284615F034F81B
:2052DC00284620F0F5FE88F4004005B0BDE8F08FB7E800205C0A0020A30E0020680E002000
:2052FC0048DD00206C0E0020A80C0020C30E002050CF00207E0E00202DE9FE4F07460868E3
:20531C000024B0B1D7E9018A0E4622F007FD8146D8F8E800082888BF0124B068204202D1CF
:20533C007068204208D003203074484622F0FEFC00242046BDE8FE8FD8F8C01069B198F8D8
:20535C00F8100029EFD006213174D8F8C410C8F8C4604E6198F8FC100DE000210522C8E9BC
:20537C003066C8E93411C8E9361198F8FC10002908BF0122327400220129726109D102201D
:20539C004FF4E02188F8FC0098F8FB001EF046F9706889490138884205D804201EF05EFA45
:2053BC0006201EF05BFA02201EF058FA98F8F80040B9DAF83C003168814203D298F8FC007A
:2053DC0000286CD0D8E9361009B118B900E028B322F0CCFBDAF80000416941F001014161D6
:2053FC00484622F0A3FC98F8F80008B10124A0E708F16C05D8F8EC10284621F00DFD00287E
:20541C00F4D0D8F8C00003210174384609F0E2F928460021002421F0FFFC8AE79AF804006B
:20543C0022F07EFC654CDAF810100222206991FAA1F1B1FA81F14368D8F8CC0040680068E3
:20545C0098472069DAF8141002224368D8F8CC0091FAA1F1B1FA81F14068006898479AF8AC
:20547C00040022F057FC9AF8040022F05BFC22F07DFB0020C8F8E000D8F8C0000068B0F5C1
:20549C00806F01D922F072FB98F8FE000028A1D1DAF80000416841F0020141609AE798F81F
:2054BC00F90020B1D8F8EC0001307FF48BAF484622F03CFCB2683AB1D8F8E8000221092883
:2054DC0038BF0121009103E008F1F40200200090746834B1D8F8E8000227092838BF012792
:2054FC0002E008F1F6040027DAF80000334D416841F002014160D6F800B0D946BBF1000F6C
:20551C0040D0D8F8E800019209284FF0010011D22A68B9F1000F1FD0C0071DD02178DAF867
:20553C0000009268904700281EBF3C44A9F101090120EDE72A68B9F1000F16D0C00714D084
:20555C002188DAF800009268904700281EBF3C44A9F101090120EDE7DAF80000D26802A90E
:20557C009047DDE90120107007E0DAF80000D26802A99047DDE9012010800098ABF1010BA5
:20559C000244BBE7D8F8F000DAF80010CA680240102802D1002AF9D101E0002AF6D0706849
:2055BC0020F0F2F8D8F8C0100020C8F8C400C8F8C00008741AE700BFFEFFFF0FC4010010F5
:2055DC002DE9F04F87B000F102098246484622F00DFB01AC06461821204621F063FD9AF81C
:2055FC00017004F10B00494622F07EFB02209AF80A108DF81A006FF00100ADF8180000205A
:20561C008DF80C0001F00800890708D480B901254FF0000B00244FF00008012115E068B92C
:20563C0003214FF001084FF0000B002500240CE0022100254FF0010B002404E0042101247E
:20565C004FF0000B00254FF000088448007838430DD0834890F8260008280BD1009121F0B5
:20567C00CDFD012F0AD148B14FF0C30B69E04FF0C30B01E04FF0C20B002464E09EB332798C
:20569C000098824218BF022F17D144EA0800012803D1D01EC0B2022807D34BEA0501501E62
:2056BC00012917D1C1B2012914D830881FF070FCD0B93088ADF8180018E04FF0000B494631
:2056DC003B468DF81AB03088ADF8180022F03AFB012437E0C0B2012802D8308822F050FB5C
:2056FC00484618F025F90026BDF818004FF6FE7188421CD11FF058FA10B1BDF818000FE09E
:20571C0027B1584C20881FF043FC30B19AF80A0000F002001CF0B8FE00E02088ADF8180085
:20573C004FF6FE71884202D14FF0C70B09E09AF80A2049463B4622F005FB002859D04FF094
:20575C00010B0024009977B1012F11D14A48007870B9002E43D0002001228DF81A0001A82B
:20577C0013F0C6FA09E001A819F0A8FD76B91AE001A83A4613F0BCFAAEB17179022F41F054
:20579C004002727104BF41F0600171719AF80A10490603D5717941F080017171B1790025F1
:2057BC000131B17100E00125B0FA80F149090C421CD107D1002C18BF834641F20100594654
:2057DC0014F0B1FD15B9484618F0B2F8BDF818004FF6FE71884218BF22F0D2FA06E00220E5
:2057FC0001228DF81A0001A813F082FA07B0BDE8F08F1D48016811B1BDF818008847BDF8E7
:20581C001800009A494605F043FB0646174818490A6800784FF4803122F015FA012115486E
:20583C00C17036B1022F0DD00099012F0FD110200AE04FF6FE7000244FF0010B0026ADF876
:20585C0018007FE7009908207279104370714FF0000B01248DF81AB075E700BF7C0B00204E
:20587C0048DD0020600E0020F0090020BAE8002098970200600C0020A80C00202DE9F04F78
:20589C008DB0044600209A4616460F46CDE90B00CDE909008748856880460FF073FF2628F3
:2058BC0003D00FF06FFF25281BD1308840F60201884218BFB0F5C15F03D1F07B022810D9AA
:2058DC003EE043F6070188420BD196F82400032807D33069784940F0806020F0604088420C
:2058FC002ED100206FB366B3387825FA00F0C00726D03046002122F035FA7048C4E9017602
:20591C00006880B109A800900CA90BAA0AAB304609F07EF80B980B214FF6FF72502320F085
:20593C006DF9FF280CD022F0F9F9654F06467878012802D840B1012070E0304622F0F6F912
:20595C0000200DB0BDE8F08F09F046FE5D480DF10409016841F0020101605B48C8F80000DC
:20597C00484621F043FDDFF864B15A494A469BF801009BF800500390554828301AF0B4F957
:20599C00554856494A461AF0AFF9484621F04EFCDFF84C81534A19214B46029540461BF050
:2059BC0021F9514A08F11C001A214B461BF01AF94E484F4922F0EEF84E484F4922F0EAF8CF
:2059DC004E48006810F4402F06D04D4A07F12800042100231FF04CFD9BF8020010B10D208A
:2059FC000FF06EF808F1400021F0B3F808F1380021F0AFF84349002007223876B8843862EF
:205A1C00386181F860200521C7E902103E49F96138700420002120F0C1F978782C4941F8BA
:205A3C00204001307870304622F080F9BAF1000F06D10DF1040A35492022504622F024FAAD
:205A5C00DAE90012BAF81000DAE90635002AB2FA82F608BF40F6C4126261216060832563C5
:205A7C00760926764FF4FA76C4E9036201226276274AC4E90722C4E90923DAF80C0000B180
:205A9C002062DAF8140000B16062DAF8080000B1E06104F13800C82121F004FB04F15000D8
:205ABC0000211FF088FB1B4904F1B80022F072F8204646E7CC2108400F000005040D00207D
:205ADC009005002000200940110000E0B4960200F8050020B162020018E10020E53B0100E3
:205AFC00B806002021C1010089A5010054E00020B154020010E000205D620200B44F00501B
:205B1C00F9EA0100C0DD002011F90000789402009B2F01008D7C02002DE9F04F8DB00646FC
:205B3C00806A447874B18D4909788C4280F012818B49023022462AB130F8023B013A21F854
:205B5C00023BF8E78748C18A708988422FD183480078A04240F2FE80B589814A214628467D
:205B7C0020F0ECFB284615F037FF064682480778BE4204D14FF6FE7015F02EFF0646BE42CE
:205B9C0080F0E880DFF8F48108EBC6094F4657F8040F08B122F0EAF8002C00F0B1806000B2
:205BBC0022F0E6F80028386040F0AC80D2E0B27C002A00F0CF806A4F0025AC4205D037F8A4
:205BDC0015208A4203D00135F7E7A04600E0A846002113F08DF9002800F0AD80814640799E
:205BFC00012840F0A88099F8060010F0180F00F0A280B9F80210204620F08EFCA54202D3B9
:205C1C00002800F098805848CDE90498B6F80C904FF6FE7A00780890544800780A90002061
:205C3C0006960B9052481130099052480430079000200C90DDE909564FF0000BF6B135F839
:205C5C00117C574518BF4F4502D1013E1C35F5E72046394620F060FC0028F6D1287801383C
:205C7C000528F2D80C980BF1010BC007EDD00B985FFA8BF1C0B28142E7D356E0DDE90786F1
:205C9C002EB338F8047C574518BF4F4503D1013E08F12408F4E72046394620F03DFC0028E7
:205CBC00F5D198F8050001380528F0D898F8000001380228EBD30C980BF1010BC007E6D065
:205CDC000B985FFA8BF1C0B28142E0D32DE00B98000628D15FEA0B6025D001205FFA8BF5F6
:205CFC000B90012D4FF001000C90A3D021F0DEFEC0B2B0FBF5F101FB15000B90012098E734
:205D1C00002038601E4989F80140A9F80250097808F83610F4B1E8B1114962000DB0BDE870
:205D3C00F04F21F003BB4FF6FE770498069EDDF8148047800A4FB37CF47CB269B18901259C
:205D5C00581EB07470895FFA88F68DE8D00003950FF010FE0DB0BDE8F08F00BFBE970200DC
:205D7C0028E6002048DD0020C9970200B797020090C5002080B40020BD970200B0AC002047
:205D9C00BC0E00202DE9F04F87B005462C200E4621F0EEFF002844D0778B044621F0B8FC3B
:205DBC000021E1840121874208BF02212170707BA0703169081A6060204617F037FB31781C
:205DDC00814F01F00301387B012908BF05206070C0B221F0FBFA4FF0FF316077A182217FC8
:205DFC00326908440A44317D3261081A3075E070A069013017D0207C032816D8DFE800F06D
:205E1C0002170209062021466082284616F04EF810B3042021466082284607F09BF80546A6
:205E3C001BE01025CBE0A32517E0A12515E00020B3256082F87A80B997F8410001280CD196
:205E5C00A07D4FF6FF7618F071FE0025A082B04208BF6FF05E0500E000252078022807D177
:205E7C0004F1080620F088FF0146304621F03CFF280640F0A180554F3878013801281AD83C
:205E9C0094F8260010B994F82700A0B1A078E178227F08441044043021F06AFF58B1A178E5
:205EBC00E2780646207F114408446168021D304621F03CFA00E0002620460DF003FD054687
:205EDC0038780138012873D8002E71D0002D6FD00DF1080800274FF0010B4FF4D00908F1D9
:205EFC00080A94F8260018B994F8270000285FD0A178E278207F114408443146021D6068D6
:205F1C0021F014FA94F8260020B184F82670C4F8129007E094F8270020B12D4884F8277060
:205F3C00C4F8120020460DF0CDFC10B10021054639E04046142121F0B5F8608A8DF819B054
:205F5C00F0B9A08A40F20311884216D0682817D16068C17B052929D12A30FF21082220F004
:205F7C0024FE18B34FF0FF306946CDE900001948006821F0B9FEFC2000E0FF208DF81800FC
:205F9C00504669460022002512F018FB01469DF8000038B10420142243461EF087FC0321E7
:205FBC00002500E0032103299BD101E00221FAE716B1304621F0DAFE204621F0D7FEE8B213
:205FDC0007B0BDE8F08F00BF48DD0020A80C0020000003010CE800202DE9FC4705460190A5
:205FFC0007788B48C65D8B48F840ADF80260C00740F00C810D2F13D1874D0DF10201A86875
:20601C00D0F8282453209047BDF802104FF6FD70814214D8019C208988B14FF0000A9CE09A
:20603C000C2F0ED0072F13D0052F0ED1A878012800F0EC80287C304400F1240916E0A8681E
:20605C00BCE06868C08AC0050AD44FF0000A09E0A87848B1A87D00EBC00006EB800905E051
:20607C004FF0010AB14605E006F11B09ADF802904FF0000A48461FF0A1F900B30446072FD9
:20609C003CD12878207068786070A878A0700028E978E170D5F8051061604FD0A87D0028DE
:2060BC00207241D0A96900293ED000EBC00004F110068200304621F039F9E66037E00C2F4F
:2060DC0040F0A4802C4654F8040F002800F09E8021F024FE804650488068D0F8541320463B
:2060FC00884748461FF06AF90446404621F01EFE002C00F08B8021F084FC2EE021F081FC64
:20611C00052F2AD104F1180561682422284621F00DF96169227C04F13C00656021F006F920
:20613C0060682430606118E000202072E060A86998B121F01BFE0020A8750DE01B2004F19E
:20615C0010061B2220723046A96921F0EFF8E660A86921F00BFE0020A8613048016819B179
:20617C0020468847002846D10D2F2CD10198426811788B0720D452783F2A1DD8284AC1F3B6
:20619C008301927C914217D190F83000022813D194F8470004F146011CF0F4FE01984FF6E5
:2061BC00FF72418E91421ED14068807902281AD3204618F0D3FA48B317488068D0F854135D
:2061DC0001A8884722E00C2F0DD1019840781A2809D0606838B1C08AC00704D0207C04F17D
:2061FC000F011CF0CFFEBAF1000F04D10D482146007817F079FC0C2F08D1019850F8041F43
:20621C0021B105498968D1F85413DAE7BDE8FC87D895020019C206000C0100203C0E002051
:20623C0048DD0020BAE800202DE9F04F93B004461DF0B0F808B11120D6E0207F4FF6FE75AD
:20625C00C0B187480078810041EA401061882077FF201EF011FE002190B1E08A05F10109E6
:20627C004FF0010B40F00400E082207F40F00100207709E04FF0000B00254FF6FE7909E0BD
:20629C004FF0000B4FF6FE7976480078022838BF01218D01678838461AF048FE08B100203F
:2062BC00607694F81AA0BAF1000F04D16E4890F800A084F81AA094F90000C6B2B0F1FF3F1F
:2062DC0007DDE07E40B969480178E1760131017002E006F00306267064490495C87A3043D1
:2062FC0004D1207E012804BF00202076DFF8748198F80000012833D8887B800730D5BBF1A2
:20631C00000F1CD0E08A410606D5BAF1010F03D120F00400E08222E0A188E07E627DADF8C8
:20633C0022708DF82AA0ADF824108DF82B0006A803F08CFC00283FF47EAF26780FE038461B
:20635C001AF0F4FD58B1002EDCD0206900780A2805D8012101FA00F010F4836FD2D1434901
:20637C004FF6FE75012E07D120690078022803D1E08A40F04000E08298F80000012806D870
:20639C00BBF1000F04BFE08A10F040002FD088460DF11701204605F0F3F806461FFA89F0B2
:2063BC00A84208BFB4F80290EEB12078617D94F82C70B8F816209DF8173007948DF818009B
:2063DC00608DADF81A00E08A06ACCDE90274CDE900101FFA89F130460BF0C0F9102803D11E
:2063FC00304621F0C3FC102013B0BDE8F08F887B88468007CCD5049EA71D6188607E3A467E
:20641C00334612F0A9FA28B100206076E08A40F02000E082387870B1618804F108001BF095
:20643C0075FA81466088814504BF00203870E08A40F04000E0822078012804D0A1886088EF
:20645C0032460EF0F5FDA188608832460CF09CFB00289DD0E08A40F02000E08298E700BFAD
:20647C00A10E0020A80C0020B197020048DD00202DE9F04F99B012AF884604461C21914643
:20649C00384620F00FFE204639460BF0B7FA9DF8550010B99DF85C0038B19DF84800410603
:2064BC000AD560891AF042FD20B140F235100FF0BCF9EDE09DF84800C0F3401A00F00C06FA
:2064DC0010F0200F18BF042E21D1E08D9DF8483010F080010CD15A060AD59DF849209207C8
:2064FC0006D143F0040202F00C020C2A40F0D3800025012213F0030320D0012B4DD0022B00
:20651C0040F0C680A08912A91AF0F6F9C0E0A58921F0FEF8854202D1E08D010609D4A5891E
:20653C0021F0F6F8854200F09280E08D010600F18E80000600F18080A08981E0DFF85CB19F
:20655C009BF80B30012B02D1A379002B7CD00223A7898DF84430ADF83C7099BB042E79D150
:20657C00207C514E8DF85E003068002800F0908021F0CEF8874240F08B80E08D217994F8B3
:20659C00302036682B460492CDE9001ACDE902900FA812A94246B0477AE0002918BF012165
:2065BC0052EA010003D1A08912A913F055FDA0890797ADF81800A0798DF81A0006A818F083
:2065DC009DF965E0ADF8300016989DF84A109DF84B208DF8203094F832300B9060898DF886
:2065FC002310DDF84E108DF8222094F830208DF83830ADF81800BBF82400CDF826109DF865
:20661C005C108DF83720ADF82400207CADF82A10A17C8DF8320020798DF834109DF85F1098
:20663C008DF833009DF85D008DF836108DF8350006A802F0E3F82BE0A089ADF86200608970
:20665C0012A91CF05BFF10B14FF49A702FE74FF0010A3AE71AB912A9384613F0FDFC11480D
:20667C000078022807D10E480078012803D1204610F000FD60B1A07CE17CBBF8242043464C
:20669C00CDE9001ACDE9029012A80FA90EF0B8F819B0BDE8F08F012500222BE748DD00201A
:2066BC00C30E0020A80C00206C0A00202DE9F04F95B0074680690DF1530200214FF0000AD6
:2066DC0004789C200AF02EFD81480078012809D8002004211BF0A4FD9DF853105FFA80FA3A
:2066FC00014400E00121C8B24FF000088DF85310A0427ED90D1B0221E8B2022828BF0D460C
:20671C001A206843C0B221F033FB0026002800F0CB80059709A95FFA85F983464FF0000809
:20673C00049006940431CDE9075102255FFA88F0484561D2E0B2824561D91EF049FA002808
:20675C0053D064490746888C393121F035F84FF60270ABF8170038888DF82460ABF8120055
:20677C00ADF82600B97A8BF8191009A811F0E6FA01460BF10A00012903D1089921F0B4FA16
:20679C0003E04FF0FF3141600160387978B1514991F83810013102288BF8181019D8012823
:2067BC008BF814501AD18BF81560012019E0494890F838008BF81550398800290A4618BF8F
:2067DC0001228BF8142018BF411E8BF81810002007E0012103288BF81410E4D001208BF88F
:2067FC0015008BF816000BF11A0B013408F101089CE70025002657E0DDF81C8005E006987E
:20681C00824534BFA0EB0A04002432480DAD4FF0020AAE1C00F139075FFA88F048453DD2FE
:20683C00E1B287202A460AF07DFCBDF83E00394620F0C2FF0BF10A00314621F055FABDF84A
:20685C0034002349234B012208F10108ABF812000978022938BF022293F838308BF81520C2
:20687C00A3F1010238BF4FF0FF3202294FF000018BF8182038BF01218BF817A049008BF8B9
:20689C001610002818BF01209DF846108BF8140001348BF819100BF11A0BBDE7DDE904673D
:2068BC00069C079D4FF00008787CE9B29DF853300022CDE90268CDE90041B91C09F00CFF76
:2068DC0016B1304621F052FA15B0BDE8F08F00BFA80C002048DD0020B0B5794C20780E2849
:2068FC0045D8DFE800F0E44444530844444444444D440808080074480078D8B1A0780328E4
:20691C004CD0012840F09880E0780130E070C0B2032800F28B806F484FF6FF71808C884219
:20693C0000F088806A48012101704FF44170A4F8010081E06A480021E170017000201BF04C
:20695C0013FE18B120780D38012851D85F480078022803D10820012104F02AF905201FF060
:20697C006DFA42F21070BDE8B0401EF0EDBD15F067F85C4810210078BDE8B04016F028BD62
:20699C005048008800F007000128B4D14E48007890B10020BDE8B04019F056BB4B480078ED
:2069BC00022849D14A480121017003200021A070484880F826103FE04A481021007816F060
:2069DC0007FD00201BF0D0FD404D0028297848D02078012950D80A284ED13A48008800F0FC
:2069FC000700022857D03B48082180F8261052E006201FF023FA334CA078000704D54FF48B
:206A1C000040012104F0D4F830480078012809D8208800F00700022804D00020002100223E
:206A3C0020F034FCBDE8B04015F00AB82A480078012801D10020A07018F07AFE1FF0AEF854
:206A5C0020488078000703D52448007801282ED1A07803282BD108200121BDE8B04004F0BD
:206A7C00A7B8022903D10820012104F0A1F805201FF0E4F901208DE703280CD114F0E0FF34
:206A9C0019480078022806D101201EF009FA02200121FDF711FE06201FF0D0F928780128C0
:206ABC0005D80848008800F00700022800D1B0BD002000210022BDE8B04020F0E7BB00BF3D
:206ADC007C0A00205EE70020DDE80020A80C0020C0E8002048DD0020B5E80020A80E002036
:206AFC003A080020BBE8002034E800202DE9F0478AB0DFF8C0810446D8F80000416E02A807
:206B1C008847DFF8B4A1DAF80800016C096811B9D0F84C058047694801210170DAF80C00DA
:206B3C00C068007830B9DAF808000021D0F858240120904720F079FF476805893878C0F351
:206B5C00401128460EF076FBDFF874910790D9F8101019B120F069FF0C308847D9F8080061
:206B7C0008B18047089057480078F0B1D9F82010B9B1884755490028554B0A4608BF02323E
:206B9C0012781A708DF82420CA1C002818BF4A1C10788DF825004C481978022908BF023036
:206BBC0000E0494801880131018014F0B1FF4A48484E0078F57350B120F037FF007D30B1AB
:206BDC00284620F0DDF91DF03DFD00286BD000253761758021F0A2F807467580059524B18D
:206BFC00012C31D13D483E49C1613C483949027B437BC47D416045804D6002F0F00202732E
:206C1C0003F0F0020232427304F0F0020432C2754A7B22F00F02531C4B73DAF808301B6C91
:206C3C001C6864682478A40608D52E4C42F002024C601B685B689B784A73A3732A4E7060F5
:206C5C00707B00F0F00070732848D8F800100822274B0C6D00210068CDE9002102AA314682
:206C7C00A0472449B0F1FF3F088007DD224819490160224801780131017010E0D9F80040A5
:206C9C0044B1DAF80800002100220023006C00680C30A047012041F2883113F019FA38460B
:206CBC0021F044F802E0E12009F0F2FF0AB0BDE8F08700BF5CE800200C010020910E0020B9
:206CDC0054930200A40B0020CCE60020DEE70020C8E80020E0E500207D0E002010E40020B5
:206CFC00801A060068E60020EC0B0020B80D00200D790000ACE80020A80B0020A10B002095
:206D1C002DE9F04F93B01C9C08901D4606928B4620461DF05BF8074620461DF03FF80026C0
:206D3C000790002F00F0E780002D18BF01254FF00008680100F14001BBF1000F08BF690122
:206D5C0005914FF6FE754FF00A0108BF0821049109A90431019100F108010C300391029025
:206D7C00380600F0C380207C804580F0BF8004EBC80B9BF81C00C00740F0B28060480078BC
:206D9C00012802D89BF81600D8B34FF0000A9BF816000F96CDE90D6678B15A49BBF8180049
:206DBC0091F86810012923D1FF21ADF83400039841F208098BF81A103EE0BBF81800A84240
:206DDC0036D104208DF824009BF81D00ADF8300009A817F0BBFD089C01980021002200232B
:206DFC00ADF83450A58015F0E7FEDDE9049024E0089C4FF00C09A080681CADF834000298D2
:206E1C001BE0BBF8180020F08DFE0028BDD0007940F002000328B8D19BF81C0040F0800082
:206E3C008BF81C00079800065DD04FF0010AAEE7ADF83400DDE90490089C8DF83600012033
:206E5C008DF83900207D8DF838000DA807F054FD9DF8480078BB109806994176417DA0F89D
:206E7C0016908BF81B109BF8161019B1254991F8681001771C9A51890185518A4185117DF3
:206E9C0080F82C10517980F83A109BF81A1080F83B102189A0F84010617D80F8491062680B
:206EBC002169C263406C227D20F040FA0DA819F0FDFE9DF848009BF81C1041F001028BF866
:206EDC001C2020B141F009008BF81C0004E00798013FA0EB0A0007901C9C4FF6FE7500262B
:206EFC0008F101083CE700200790F9E72046002116F070F80646304613B0BDE8F08F00BF5D
:206F1C00A80C002048DD00202DE9F04F8BB0002900F0F080DDF858A00746007A0D4699465D
:206F3C0090465FEA0A718DF8060012D4387A02240F2800F2E0800121814011F00B0F19D0E2
:206F5C0003288DF8100024D102A8394620F0CCFE22E0022840F0CE803C8820F0D9FB844245
:206F7C00E4D038880121032212F086FF0028DDD0CD24C0E048F20400014200F0BC803888E0
:206F9C0019F0D4FF002800F0B1800F2038728DF810003888ADF808005FEA8A7014D400208A
:206FBC00ADF818005648006888B14168A942FAD1826862B129780220904768B10188ADF87C
:206FDC00181020F0D3FE07E04FF6FF7002E0A86810B14088ADF8180000205FEACA61ADF880
:206FFC00200009D59DF810100020012904D00F291CBF0420ADF820001021CAF38013DDE961
:20701C00142B01EADA011AF0C00F08440AF0400140EA911018BFADF820008DF805305FEA85
:20703C004A73179944BF4030ADF820000792ADF81A90ADF8168000208DF824107C7A7E8996
:20705C008DF804009BF800005FEA8A612D498DF81340ADF814608DF82200287809788DF810
:20707C00120048BF04218DF823101FF053FC28B1016919B102A888477C7A7E893046214640
:20709C0020F0E2FB28B11FF059FE48450DD2022413E001A81FF02EFF48450AD21A4801680A
:2070BC000029F4D002A8884706E002A806F0D4FD02E002A801F0A2FB04469DF810000228C4
:2070DC000CD1BDF8086020F023FB864206D19BF800102878424623461AF0DAFD5CB99BF810
:2070FC000000002401308BF8000004E0387A0F287FF426AF022420460BB0BDE8F08F00BF5D
:20711C004CE8002037040020D80D0020BFB581780446481E0B2812D8DFE800F006525C6A90
:20713C0026788590A430B23900208DF80400E0780F28C0F0B28002208DF80400B3E0FF2941
:20715C0040F0D3800025E01C04218DF803501DF045FC6C4908606C48058010F087FF0DF14A
:20717C0003036F20FF21BDE000208DF80800E07801F0CAFE02AB6F200521B3E01EF08EFE54
:20719C008DF80E000DF10E036F200A21AAE000208DF80F00E01C20F0E7FD0546601D04215C
:2071BC001DF01CFC014628460CF02AFB504A3520282120F0C7FB0DF10F036F200C2191E071
:2071DC0000208DF80600E0780F2870D302208DF8060072E0E07847490DF10703002818BF28
:2071FC0001200870002003218DF807006F2079E0E2780020211D8DF80A0004F10C00022AAE
:20721C0068D0012A6AD116F0FBFD65E000208DF80C00E078002818BF01201FF0FFF803AB94
:20723C006F2006215EE0E078211D18F005F98DF80D000DF10D036F20072153E00020E5789B
:20725C0004218DF80900201D1DF0C8FB002D014618BF012528461FF06BFE0DF109036F2062
:20727C0008213FE000208DF80B00E078002818BF012020F019FB0DF10B036F20092131E088
:20729C0000208DF80500E07804281BD21B4A01211070512020F056FB17E0194A01211070E2
:2072BC00522020F04FFB01AB6F2001211AE0124A01211070532020F045FB0DF106036F2038
:2072DC0002210FE002208DF805000DF105036F200B2107E00AF0D2F98DF80A000DF10A03CD
:2072FC006F200421012219F0E1FD002004B0B0BD80E300209C0E0020B00E0020BA0E002060
:20731C00B60E0020900B00208C0B00202DE9F04F8BB0846906462588B4F80290284619F0D0
:20733C0005FE01280DD1307C717C00228023CDE90052CDE90220B21C48F2060016F008FDD0
:20735C00D1E0284619F0F2FD20B96A480088854240F0C48008962679651D5EB1700020F05E
:20737C0007FD38B10246304629460A921FF0F0FE054602E0002000260A9015F8017B57B1A0
:20739C00780020F0F5FC30B102463846294609921FF0DEFE02E0002000270990B8191421F4
:2073BC00DFF858B14FF6FF754FF0000801EB4000C0B207907800069070000590DBF800B006
:2073DC00BBF1000F66D0DBF8040001780029F5D09BF80E20D207F1D0DBF808401CB10120FE
:2073FC00A047824601E0D0F808A0BAF1000FE5D0BAF80200814518BFA94545D1DAF80830A3
:20741C009AF807200A9930461CF02AFE40B9DAF810309AF80C20099938461CF021FE98B3EB
:20743C0007981DF0CBFF28B30546D2202870089840882F732E7168803EB10A99059A05F152
:20745C001400A8601FF072FF01E00020A86047B105EB46000999069A143028611FF066FFBA
:20747C0001E000202861DBF8040029464068007816F03AFB9AF80000214A5FFA88F108F1FD
:20749C0001084FF6FF755054002C97D0504620F06DFC93E7089C0A9D5FEA086011D0154814
:2074BC005FFA88F3227C617C0088CDE9000314480023CDE90202A21C48F2060016F048FC9F
:2074DC0001E0207B90B115B1284620F04FFC099848B10BB0BDE8F04F20F048BC0648007831
:2074FC0002283FF420AF0BB0BDE8F08F4FF00008D5E700BFA8E70020A80C00204CE80020CC
:20751C0004E2002070B590B0044680781FF03EFA002800F0CF8005466078A0F1E101E87303
:20753C00102906D91A2818BFCD2808D01D2806D04BE0012202FA01F16A4A1142F2D06A4E59
:20755C003078012802D8688900056CD42846002107F0AEFEC0B3307801282BD86348807B0F
:20757C00800727D52968086A20B3C97F03AA08F0C3FE6078E92808D12868E27B012341894B
:20759C0000880093E92301F04FF82868BDF8161001809DF81120BDF81810BDF81600002AEC
:2075BC0018BF012292010BF0EFFA18B1688940F0200068816A89617828891EF0FFFC28811C
:2075DC003078012831D96DE060788DF81000A07B03958DF81100287C00283ED003A811F02B
:2075FC0047FF9DF81030E92B00D03BB92868E27B012641890088009601F016F83A48007887
:20761C0001284FD83948807B80074BD5687B022802D16889400737D46078E92842D128464E
:20763C0019F0A4FF3EE0052068736078E92839D02F48006800B180472E4E306890B32B4851
:20765C00807B80072ED52868418900881AF02EFC40B361783268904724E003A805F026F874
:20767C0021489DF8103000780128BCD8002BBAD12868008819F05AFC0028B2D11C480068D7
:20769C000028AED08047ACE72868008819F04EFC002811BF032028684FF6FF71018008BFBB
:2076BC0005206873687B022804BF06206873A07811F09EFD1DF0B8FD0B48007802280ED193
:2076DC000D48007858B900200DF10B018DF80B00522019F0EFF82020012103F069FA10B01C
:2076FC0070BD00BF01010100A80C002048DD0020D4090020D8090020C30E0020DFF8DC8143
:20771C00774F784DDFF8E0A1DFF8E0B14FF00009D8F800004FF0FF3120F000FD1FF0F4FC6F
:20773C00B9783A792C68BB7987F8029087F8049087F80690002918BF44F00404002A18BF0B
:20775C0044F08004002B18BF44F002042C601FF045FB2868010644BF20F0800028609AF8FA
:20777C00000015F007FE00283FD0F968044649B17878012804D0022804D12046884734E0D2
:20779C0020468847204614F0E2FE70B304460C2020F0EEFA88B10646D1461FF0B5FC824699
:2077BC002078B46080B1304620F0E0FA60681EF07FFC204620F0DAFA11E060681EF078FC9A
:2077DC00204620F0D3FA10E0DBF80000314620F0A1FC286840F01000286020F0BBF95046B1
:2077FC001FF0FCFACA464FF000092868C1062BD520F0C8F9E8B91FF0AFFFD0B91FF084FC72
:20781C000446DBF8000020F081FC78B1064680684188406815F080F8B06840681EF048FC45
:20783C00B06820F0A3FA304620F0A0FA20461FF0D5FA20F0A7F920B1286820F0100028604A
:20785C0002E020F087F9286881070CD506F0E8FC1EF0E4F918B120F07DF9286803E028688A
:20787C0020F002002860010722D5DBF8040020F04DFC80B1B968044639B1387828B10228EA
:20789C0028D0012804D1A0688847A06818F030F9204620F06BFADBF8040020F033FC20B104
:2078BC00286820F00800286002E020F053F9286841077FF52DAF20F00400286020F062F90F
:2078DC0000287FF425AF286840F01000286020F041F91DE7A0688847DAE700BF78E80020A0
:2078FC00BC0B00207CE80020DBE80020B40C00202DE9F843DFF8B8810546894601211F463C
:20791C001646D8F80C00C06801706A480021017069480170D8F80800016C096811B9D0F8CC
:20793C004C058047654804684CB1654832463B464188D8F80800006C00680C30A04717F0B8
:20795C00E24F14D05F480178013901705C48406810B15D4820F0F6F8D8F80800006C0068CF
:20797C004068007880066BD41CF01CFF6BE030070BD45348406810B1534820F0E3F851485B
:20799C000178013901701D205BE04E4E4F4F42F20541307801383070788840F004008842FC
:2079BC0011D14748406810B1474820F0CBF8484849460068826C2846904720B1008842F624
:2079DC000141884254D13E4842F606024188914212D0B1F5105F43D140694149086019F049
:2079FC00A5FD3C48007870B33C480168013118BF01600021018126E0406810B1324820F0B7
:207A1C00A1F834480078F0B133482F4900780A1D022808BF8A1D10884FF0040200F1010023
:207A3C0008BF062288522D484168013118BF41600189428901318BB20181934288BF418175
:207A5C00E92009F025F91F48017819B390F90000002826DCD8F80800D0F84C05804720E0D3
:207A7C00406800283FF48FAF174820F06BF88AE7154842F205424189013141817988E120CE
:207A9C00914208BF1C2009F003F9307810B196F90000DDE7D8F808000021D0F858240020E6
:207ABC009047D8F80C000021C0680170BDE8F8830C0100209F0B0020910E0020549302007E
:207ADC00E0E50020A10B0020CCE6002010E400205CE80020A40B0020C8E8002084E7002065
:207AFC0070E800202DE9F04788B004464FF0FF3002214FF6FE79CDE90200E089002808BFC6
:207B1C000821A66916F801A030B16C4835880088854210D16A4E06E0694831461DF04AFFC4
:207B3C0060B36648058800214D4518BF002E42D06548406845E06348007801281CD82846E9
:207B5C001FF0F0FFC0B10179002601292AD140880DF110088DF81060ADF81C00404616F0B5
:207B7C00F5FE0646002818BF08F10406BAF1000F18BF4FF0FF3AD6E7002613E051480078B8
:207B9C0001280DD8304620F031F848B101790139012905D8BAF1000F18BF4FF0FF3AC1E7A7
:207BBC004FF6FE75B5EB0900314618BF0120002E18BF01210140207B00287BD14248406830
:207BDC0051B15FFA8AF1022901D200270DE0217B01296FD0802708E0E189812719B100F839
:207BFC00017B02AE04E009F1010500F8017B0EB1314600E002A920F077F80570064605805F
:207C1C0030484FF00B080078012844D8002F42D15FFA8AF001283ED12848A9B2008881425E
:207C3C0039D100250DF107008DF8075015F060FA98B1E1890322002908BF0922A1698B5CD5
:207C5C009DF8072000EB43019A420AD9D21A0D258DF8072005EB420808E04FF00C08B570FA
:207C7C0019E000224FF00D088DF80720F370331DB27012060DD011F8022B03F8022B11F89C
:207C9C00012C03F8012C9DF80720013A8DF80720EFE720F06BF8E2890B4D1020A11C5FFA7E
:207CBC0088F3A87004F1110042F4004216F000F90020A87008B0BDE8F08700BFA8E700201E
:207CDC0000E80020A80C00200C0D00202DE9FE4F1D4614460F46814620F020F8DFF8BCA1DB
